:100000000C94C3090C94EB090C94EB090C94EB09C8
:100010000C94EB090C94EB090C94EB090C94EB0990
:100020000C94EB090C94EB090C94EB1F0C945A20E4
:100030000C94EB090C94EB090C94EB090C94EB0970
:100040000C94EB090C94EB090C94EB090C94EB0960
:100050000C94EB090C94EB090C94EB090C948C2296
:100060000C94EB090C94EB090C94EB090C94EB0940
:100070000C94EB090C94EB090C94EB090C94EB0930
:100080000C94D6220C94EB090C94EB090C94EB091C
:100090000C94EB090C94EB090C94EB090C94EB0910
:1000A0000C94EB090C94EB090C94EB090000000094
:1000B000F87FF87FFCFF4CC2FCFF54BAFCFF5CBA2F
:1000C000FCFF5CBAFCFF5CA0FCFF5CACFCFF5CAC22
:1000D000FCFF5CA0FCFF5CBAFCFF5CBAFCFF54BAFE
:1000E000FCFF4CC2F87FF87F000000000000000019
:1000F0000000000000000000F007F007F047F047A4
:10010000F087B086F007B006FCFFB4F6FCFFB4F64B
:10011000F007B006F087B086F047F047F007F00729
:1001200000000000000000000000000000000000CF
:10013000000000000000000000380038007C00448F
:1001400038FE38BAF8FFE8BDFCFF0CBCFCFF0CBC65
:10015000F8FFE8BD38FE38BA007C004400380038AB
:10016000000000000000000000000000000000008F
:1001700060006000E00FE00DF03FF03DF17FF17DA9
:10018000FBFFFBFDFFFFFEFDFFFFFEFDFFFFFEFD92
:10019000FFFFFEFDFBFFFBFDF17FF17DF03FF03D3A
:1001A000E00FE00D60006000000000000020000093
:1001B000007000000070000000F80000C0FFC03FA9
:1001C00000F9000900F9000900F9000900F9000927
:1001D00000F9000900F90009C0FFC03F00F8000065
:1001E000007000000070000000200000040000000B
:1001F0000E0000000E0000001F000000FF03FC03C3
:100200009F0090009F0090009F0090009F00900032
:100210009F0090009F009000FF03FC031F00000060
:100220000E0000000E0000000400000001000200AB
:1002300004000800100020004000800000010002BF
:1002400000040008001000200040008001020408A3
:10025000102040800F00080F0004080C0F0002055A
:10026000080A0D0F00020406080A0C0E0F00010315
:10027000040608090B0C0E0F00010204050608090C
:100280000A0C0D0E0F0001020304050608090A0BF3
:100290000C0D0E0F000102030405060708090A0BE6
:1002A0000C0D0E0F0F0000010203040506070808DD
:1002B000090A0B0C0D0E0F0F0000010203040405C8
:1002C00006070808090A0B0C0C0D0E0F0F000001A1
:1002D00002020304050506070808090A0A0B0C0DAB
:1002E0000D0E0F0F000001020203040405060607AD
:1002F0000808090A0A0B0C0C0D0E0E0F0F00000166
:1003000001020303040405060607080809090A0B8D
:100310000B0C0C0D0E0E0F0F000001010202030466
:10032000040505060607080809090A0A0B0C0C0D46
:100330000D0E0E0F0F00000101020203030404055D
:1003400005060607080809090A0A0B0B0C0C0D0D17
:100350000E0E0F0F00000101020203030404050545
:1003600006060707080809090A0A0B0B0C0C0D0DF5
:100370000E0E0F0F0F190D320414030200600099C6
:100380000C1E05140302016000190C14070A020078
:10039000005001990B0A07050100003200FFFFFF22
:1003A000FFFFD1FFFFF9FFF9FFC1EBC1FFD3C1E5AB
:1003B000FFCDF7D9FFCBD5EBFFFFF9FFFFFFE3DD63
:1003C000FFFFDDE3FFEBF7EBFFF7E3F7FFDFEFFF07
:1003D000FFF7F7F7FFFFDFFFFFCFF7F9FFC3DDE11F
:1003E000FFDBC1DFFFCDD5D3FFDDD5EBFFE1EFC7ED
:1003F000FFD1D5E5FFC3D5E5FFCDF5F9FFC3D5E1C5
:10040000FFD3D5E1FFFFEBFFFFDFEBFFFFF7EBDDF6
:10041000FFEBEBEBFFDDEBF7FFFDD5F9FFE3DDD302
:10042000FFC3F5C1FFC3D5E9FFE3DDDDFFC1DDE3B8
:10043000FFC3D5D5FFC3F5F5FFE3DDC5FFC1F7C1A8
:10044000FFDDC1DDFFEFDDE1FFC1F7C9FFC1DFDF88
:10045000FFC1FBC1FFC1FDC3FFE3DDE3FFC1F5F356
:10046000FFE3CDC1FFC3F5C9FFDBD5EDFFFDC1FD46
:10047000FFE1DFC1FFE1DFE1FFC1EFC1FFC9F7C964
:10048000FFF9C7F9FFCDD5D9FFFFC1DDFFF9F7CFE0
:10049000FFFFDDC1FFFBFDFBFFDFDFDFFFFFFDFB3C
:1004A000FFE7DBC3FFC1DBE7FFE7DBDBFFE7DBC128
:1004B000FFE7CBD3FFC3EDFBFFB7ABC7FFC1F7CF60
:1004C000FFFFE5DFFFBFCBFFFFC1F7CBFFFFE1DFA2
:1004D000FFC3F7C3FFC3FBC7FFE7DBE7FF83DBE730
:1004E000FFE7DB83FFC3F7FBFFD7D3EBFFE1DBDFE6
:1004F000FFE3DFC3FFC3DFE3FFC3EFC3FFCBF7CBF4
:10050000FFF3AFC3FFDBCBD3FFF7C1DDFFFFC1FFBD
:10051000FFDDC1F7FFFBFDFBFFE3EDE3FFD5F08D52
:1005200014A1C881CFD9F1AF20003101070000002C
:1005300015008D010700000007003C0307001902A9
:100540000700380207005A020700800007005A021D
:100550001D007E0007005A0207003802070028022B
:100560000700190207007D000E008D010700280119
:10057000070020010700F8000700EF0007007D00DA
:100580000700AC0007009B000700930007008E00E7
:1005900007008B00070087000700840007007D002C
:1005A0000700810007000080466F756E6420616E51
:1005B00020616E6369656E74207363726F6C6C008A
:1005C000466F756E642061206A6577656C20656E84
:1005D000637275737465642063726F776E00466F23
:1005E000756E6420736F6D6520676F6C6420636F38
:1005F000696E73004472616E6B206120706F746964
:100600006F6E206F66206865616C696E670095018A
:100610000700000015008D01070000000700160408
:1006200007007F00070000000E00770107000000B0
:100630001D0046010700400107003B0107000000C4
:100640004700E7000700E4000700000015009F00D6
:1006500007009D0007000000880088000700008058
:1006600051010700000015008D0107000000070080
:100670004B0107003601070046010700690107002A
:100680009E0107007F000700850107002802070080
:100690006D020700FC020700E0020700FD010700F1
:1006A000190207003C030700E7000700810207006A
:1006B0006D020E002D050E00DA040E001C0107006D
:1006C00087030700600307003C0307008703070058
:1006D000AD020E00C60207000C010E00E00207008A
:1006E000C602070096020E0081020700AD02070055
:1006F000C6020700E0020700E10007001B03070035
:100700004802070019020700F1010700D9010E0095
:10071000F10107000B020700AD020700D10007003E
:1007200048020700380207001902070028020E00DD
:100730000B020700E5010700D90107000080E00275
:10074000070000001500E203070000000700DA04BC
:100750001500B4000700D901070000000700F101EF
:100760000E0080000700F101070000000E005A0291
:100770000700E400070000001500C10007000000AA
:100780000E00E501070000000700AC0007000000B4
:1007900015009100070000801001070000001500FF
:1007A0008D01070000000700D9010700FD010700C7
:1007B0000B020E0028020E00380207004802070054
:1007C0006D020700810232006D0215004802070029
:1007D00038020700B00107007E0107006901070029
:1007E0004B01070036010700310107000201070035
:1007F000F8000700F2000700E9000700E400070026
:10080000D8000700BD000700AB0007009D000700EF
:100810009600070094000700920007008E00070072
:100820008B0007008A000700890007008800070086
:100830008700070086000700850007008400070086
:10084000830007008200070081000E00810007007E
:10085000800007007E0007007D0007007D00070084
:100860000000400090003200008000000000000006
:100870000000000000000000000000000000000078
:100880000000F000B000FC7F9C5EFA7F9A5EF000F2
:10089000B0000000000000000000000000000000A8
:1008A0000000000000000000000000000000000048
:1008B0000000000000000000000000000000000038
:1008C0000000F000B000F87F985EFD7F9D5EF000B4
:1008D000B000000000000000000000000000000068
:1008E000000000000000000000003E006F6666008F
:1008F0006F6E00536F756E643A00537461727400CA
:10090000627920406A616D657368686F77617264AF
:100910000043415441434F4D4253204F46205448D9
:10092000452044414D4E454400456E746572696EE4
:100930006720666C6F6F720000000000C007000047
:10094000F00F0000F81F0000FC3F0002FE3F000116
:10095000FE7F9001FE7FE003FE7FC007FE7F8009DF
:10096000FC7F8000FC3F4000F81F0000F00F0000FB
:10097000E003000000000000000000000000000094
:10098000F000F000F801F801FC03FC03FC07DC07B1
:10099000FC073C07FC173C16F8077804F02FF02CF6
:1009A000E00FE00F001E001E8018801800220022B9
:1009B00000000000000000001C1C000000000000FF
:1009C000000000000006060F0E1F1C7E78FCF4FEDF
:1009D000E8FC90F860F080E000800000000000007B
:1009E0000000000000000000000000000000000007
:1009F0000000000C0C1E1C3E387C70F8E0F0C0E0DB
:100A000080C080C080C7C7FFFFFFFFFFF8FFFFFF68
:100A1000E0FFFCFE00FC0000000000000000000001
:100A200000000000000000000000000000000000C6
:100A3000000000000003030F0F1F1F3F3F7F7FFFD9
:100A4000FFFFFFFFFFFFFFFFFFFFFFFFFEFFF0FEC7
:100A500060F040E000C000800000000000000000E6
:100A60000000000000000000000000000000000086
:100A700000000000000000000001010F010F010F45
:100A8000000F000F000F000F000F000F000F000FEE
:100A9000000F000F000F000E000C1C1B00000000D8
:100AA00000000000003838FCF8FCE0F880E000802E
:100AB00000FFFEFFFCFEC0FC00F0F0F8F0F800F0D4
:100AC000C0E000C0000000000000000000000000C6
:100AD0000000000000000000000000000000000016
:100AE0000003030F0FFFFEFFFCFFFFFFFFFFFFFFF1
:100AF000F8FFFFFFFFFFFCFFFFFF1FFF001F0000CD
:100B00000000000000000000000000000008081CB9
:100B1000183C183C183C183C183C1C3E3E7F3F7F5C
:100B20007FFF7FFF7FFFFFFFFFFF7FFF3FFF1FFF75
:100B30001FFF0FFF0EFF00FE00F000F000E000E0DE
:100B400000C000C000000000000000000000000025
:100B50000000000000000000000000000000000194
:100B60000001000700070007000700070007000753
:100B70000007000700070007000700077CCEB69AB1
:100B8000B6CE7C007CE6C68EC6E67C0046494E4169
:100B90004C2053434F52453A0000000000DC0FDC6C
:100BA0000F78004800F07F007FF8817880FC1FFC00
:100BB0001EFC277C27FC0F540FFC0F6C0FFC277CBE
:100BC00027FC1FFC1EF8817880F07F007F780048AA
:100BD00000DC0FDC0F0000000000000000B007B0D8
:100BE00007F0089008E03F003EF043F040F83FF87F
:100BF0003DF84FF84EF81FA81EF81FD81EF84FF802
:100C00004EF83FF83DF043F040E03F003EF00890E2
:100C100008B007B0070000000000000000800700D7
:100C200000C0030000E0030000C0070000C0010096
:100C300000F00F8000E0070000E0070000F00F80E8
:100C400000C0010000C0070000E0030000C0030076
:100C500000800700000000000000000000400100CC
:100C600000C0030000C007000080070000800300F0
:100C700000E01F0001C00F0000C00F0000E01F00D7
:100C8000018003000080070000C0070000C00300CF
:100C900000400100000000000000000000000E0005
:100CA0000C000F000980078003F807F803FCFF041D
:100CB00077FE3F5626FE3FF636FE3FF636FE3F569F
:100CC00036FC7F0437F803F803800180011C1E1CEA
:100CD0000CF67FF66D000000000000000000000030
:100CE00000000C000C800F800BF007F003F87F0869
:100CF00036FC3FAC24FC3FEC35FC3FEC35FC3FAC14
:100D000034F8FF0876F003F00300030003383C38A2
:100D100018ECFFECDB0000000000000000003F00CA
:100D20003F007F0041007F005D007F005DFC7F7C15
:100D300041FE7F6E3FFE3F0E00FE1F0E1BFEFF6E4C
:100D4000FBFCFF7CFB801F0011801F0004FC1FFCCC
:100D500015000E0004000E000000000000003F001F
:100D60003F007F0041007F005D007F005DF8FFF8DD
:100D7000C1FCFFDCBFFC3F1C00FC3F1C36FC7FDCE1
:100D800076F87FF876001F0002001F0008F83FF891
:100D90002B001C0008001C00004B494C4C533A002F
:100DA00000000000000000000060006000F000D0C3
:100DB00000F000D080FF80DFC07F4075C07F4075AD
:100DC000C07F4075807F807F00FC00D400FC00D491
:100DD00000FC00D400780078000000000000000053
:100DE000000000000C000C003C9C309CFCFF846F59
:100DF000FCFFFC8DFCFF5CEFFCFF5CEDFCFF7CED81
:100E0000FCFF5CEDFCFF5CEDFCFF5CEDFCFFDCED52
:100E1000FCFF5CEFFCE3FCE378607860000000001E
:100E20000000000000000000C03FC02F807E805EF8
:100E3000007C005C00FC00BC20FF20BFF0FFF0B98C
:100E4000F0FFF0B920FF20BF00FC00BC007C005C7C
:100E5000807E805EC03FC02F0000000000000000C8
:100E600000000000F07FF07FF8FF18C2F8FFE8BA3A
:100E7000F8FFF8BAF8FFF8BAF8FFF8A0F8FFF8ACF6
:100E8000F8FFF8ACF8FFF8A0F8FFF8BAF8FFF8BAE6
:100E9000F8FFE8BAF8FF18C2F07FF07F000000000A
:100EA0004C4F4F543A004B696C6C6564206279205A
:100EB0006120737069646572206F6E206C65766561
:100EC0006C004B696C6C6564206279206120626102
:100ED00074206F6E206C6576656C004B696C6C6578
:100EE000642062792061206B6E69676874206F6E80
:100EF000206C6576656C004B696C6C65642062796A
:100F00002061206D616765206F6E206C6576656C71
:100F100000596F752065736361706564207468653E
:100F20002063617461636F6D6273210047414D45B9
:100F3000204F56455200080B00020202000009042F
:100F40000000010202000005240010010524010137
:100F50000104240206052406000107058103100090
:100F60004009040100020A000000070502024000D7
:100F70000007058302400000040309041201000277
:100F8000EF0201404123368000010102030141725A
:100F90006475696E6F204C4C4300414241313330DF
:100FA00036004162616E646F6E20616C6C20686F08
:100FB00070652079652077686F20656E7465722191
:100FC00000466F756E6420612063686573742066E7
:100FD000756C6C206F662074726561737572652123
:100FE000002001070000001500E9000700000007CD
:100FF00000560115000000320085011D0000004070
:10100000000B02150000003200870324000000409E
:101010000087032B0000004000B203320000800074
:101020000006000C00120019001F0025002B0031E3
:101030000038003E0044004A00500056005C006149
:101040000067006D00730078007E00830088008ECA
:1010500000930098009D00A200A700AB00B000B56F
:1010600000B900BD00C100C500C900CD00D100D449
:1010700000D800DB00DE00E100E400E700EA00EC5D
:1010800000EE00F100F300F400F600F800F900FBB8
:1010900000FC00FD00FE00FE00FF00FF00FF00FF5F
:1010A00000FF00FF00FF00FE00FE00FD00FC00FB53
:1010B00000F900F800F600F400F300F100EE00EC97
:1010C00000EA00E700E400E100DE00DB00D800D425
:1010D00000D100CD00C900C500C100BD00B900B5F8
:1010E00000B000AB00A700A2009D00980093008E06
:1010F00000880083007E00780073006D0067006147
:10110000005C00560050004A0044003E00380031A8
:10111000002B0025001F00190012000C0006000023
:1011200000FAFFF4FFEEFFE7FFE1FFDBFFD5FFCFA3
:10113000FFC8FFC2FFBCFFB6FFB0FFAAFFA4FF9F1E
:10114000FF99FF93FF8DFF88FF82FF7DFF78FF727D
:10115000FF6DFF68FF63FF5EFF59FF55FF50FF4BB8
:10116000FF47FF43FF3FFF3BFF37FF33FF2FFF2CBE
:10117000FF28FF25FF22FF1FFF1CFF19FF16FF148A
:10118000FF12FF0FFF0DFF0CFF0AFF08FF07FF050F
:10119000FF04FF03FF02FF02FF01FF01FF01FF0148
:1011A000FF01FF01FF01FF02FF02FF03FF04FF0534
:1011B000FF07FF08FF0AFF0CFF0DFF0FFF12FF14D0
:1011C000FF16FF19FF1CFF1FFF22FF25FF28FF2C22
:1011D000FF2FFF33FF37FF3BFF3FFF43FF47FF4B2F
:1011E000FF50FF55FF59FF5EFF63FF68FF6DFF7201
:1011F000FF78FF7DFF82FF88FF8DFF93FF99FF9FA0
:10120000FFA4FFAAFFB0FFB6FFBCFFC2FFC8FFCF1D
:10121000FFD5FFDBFFE1FFE7FFEEFFF4FFFAFFCEB4
:10122000010700000015008D0107000000070016EF
:1012300004070091040700B2030700DA0407002D39
:10124000051500DA04070091040700E00207009684
:101250000207005A020700F1010700190207000007
:10126000000700CE0107007C000E005C0107007D36
:10127000000E00200107007D000E00EF000700D5E2
:10128000000700CA00070000000700C1000700B9FE
:10129000000700B3000700A90007007D0007007EDB
:1012A000000700930007007E000700000007008988
:1012B0000007008500070082000700800007007E0D
:1012C0000007007D0007000080B001070000001546
:1012D00000C800070000000700B203070060030712
:1012E00000E0020700960207004802070019020703
:1012F00000FD01070050040700CE010700B90107F7
:1013000000A7010700500407007E010700630107E2
:1013100000400107002D0507001001070009010723
:101320000002010700F8000700DA040700CA0007FE
:1013300000BB000700B300070091040700960007F8
:1013400000D800070000001D009602070000002BD7
:10135000002802070000002400FB000E00008001AE
:1013600003070F1F3F7FFFFFFEFCF8F0E0C0800582
:10137000002B802B005580552B002B2B552B5555C2
:10138000405540801D2311241FBECFEFDAE0DEBFA1
:10139000CDBF11E0A0E0B1E0E2E1F7E602C00590C8
:1013A0000D92AA32B107D9F72AE0AAE2B1E001C052
:1013B0001D92AF31B207E1F719E0C3ECD9E004C0E8
:1013C0002197FE010E943E33C23CD107C9F70E941B
:1013D00042230C9487330C9400008091C502089539
:1013E00090E0EFEBF5E091119FEF8FEF91939193E8
:1013F000919391938150D0F70895CF93DF939C01FF
:10140000EB0150E2459FC001112464E670E00E94A8
:101410002B33462FD90190E080E0FE01E80FF91F41
:10142000E491ED93019688309105B9F778E0740F57
:10143000761B6150E901C70FD11D6F3F19F0B6EC63
:10144000B883F4CF81E0870F783220F49EEF999330
:10145000782FF8CF6EEF6883D901A80FB11D1C92C9
:10146000DF91CF9108959091E203911103C08FEF26
:101470009FEF08954FB7F89422E02093E900509130
:10148000F200252F30E01216130614F421E030E0AC
:10149000232B31F0289884E68093E1038091F100BA
:1014A000552339F03091F200311103C06BE660939F
:1014B000E8004FBF5523D9F290E008952FB7F89474
:1014C00083E08093E9009091E800892F807295FF76
:1014D00004C03091F20080E4831B2FBF08958091F7
:1014E000D90381110DC022E02093D50334E030935D
:1014F000D6031092D8031092D70341E04093D9034A
:1015000085ED93E00895A1E0B0E0E9E8FAE00C94FD
:1015100060336983DC01ED91FC910280F381E02D61
:1015200041E050E0BE016F5F7F4F09952196E2E0F8
:101530000C947C3383E08093E9002091F200222315
:1015400019F03AE33093E8000895B8DF90E0089589
:10155000FC018485958597FD05C02FEF3FEF35870A
:101560002487089580CF0895CF93DF93EC018C8575
:101570009D8597FF03C077DF9D878C878C859D8530
:10158000DF91CF910895FC018485958597FD0BC06F
:101590003FB7F89442E04093E9008091F2003FBFEA
:1015A00090E0019608959FB7F89422E02093E90017
:1015B0008091F2009FBF90E008954091CF03509139
:1015C000D0032091CD033091CE0342175307B4F4DA
:1015D0009091E8009570E1F33091E80032FD19C078
:1015E0008093F1008091CF039091D00301968F7387
:1015F0009927892B19F45EEF5093E800A091CF034F
:10160000B091D0031196B093D003A093CF0381E0A3
:10161000089580E00895EF92FF920F931F93CF9368
:10162000DF93F82E192FE62E042F81E0860F880F06
:10163000C4DF83E0C2DFCF2DD12FEC0EFD2EF11CD5
:10164000CE15DF0599F007FF0FC0FE018491B5DFCD
:10165000182F80E0B2DF812321968111F1CFCDB721
:10166000DEB7E6E00C9478338881F1CF81E0F7CFE4
:10167000B0E0A0E0EEE3FBE00C945B33D82E8A01EF
:10168000EB017B01E40EF51ECE15DF0551F0D7FE10
:101690000EC0FE01849191DF21968111F5CF0FEFED
:1016A0001FEFC801CDB7DEB7E7E00C947733888130
:1016B000F2CFA1E0B0E0EFE5FBE00C945E3382E016
:1016C000898342E450E066E37FE080E8D1DF07DF12
:1016D000FC01028113810115110589F0D801ED91FA
:1016E000FC910280F381E02DBE016F5F7F4FC80146
:1016F000099597FD04C0F80100851185ECCF89811B
:101700002196E4E00C947A33615030F02091F1009E
:10171000FC0120830196F8CF289884E68093E103AA
:101720000895FC017FD0319728F068517C4F8F4F8E
:101730009F4FF9CFAB01FC0175D0641775078E0779
:101740009F07D0F30895B0E0A0E0E9EAFBE00C9435
:1017500058336C01B62EA72E7A0180910F01882391
:1017600009F453C02091E203222309F44EC00091F2
:10177000D40300FF05C01091E00012601093E00058
:10178000E70110E00AEF209711F41123B9F196DE7A
:10179000811106C00150C9F181E090E0C2DFF3CFB2
:1017A0008C171D0611F00CF08C2F9FB7F89433E0C6
:1017B0003093E9004091E80045FD02C09FBFE3CFB0
:1017C000C81BD109EB2DFA2DBE2EAF2E815020F073
:1017D000A190A092F100F8CF112329F07AE3709341
:1017E000E80010E0EBCF5091E80055FDE7CF6AE349
:1017F0006093E80011E0209709F3F3CF5D98A4E629
:10180000A093D3031E141F043CF0C1E0D0E0F60106
:10181000D383C283F12CE12CC701CDB7DEB7EAE058
:101820000C947433A9ECB3E02FB7F8947D918D91AB
:101830009C9166B52FBFA89B05C06F3F18F47F5FD2
:101840008F4F9F4F22E0660F771F881F991F2A95A1
:10185000D1F708952091B702E091B502F091B60258
:10186000CF0102969093B6028093B502222319F01D
:10187000859194910895808191810895CF92DF920E
:10188000EF92FF92CF93DF93E5DF811520E8920777
:1018900091F4909171009D7F90937100109291004E
:1018A00046985F981092B402DF91CF91FF90EF902D
:1018B000DF90CF90089521E02093B402813020E89A
:1018C000920749F48091B2029091B3029093B602CC
:1018D0008093B502BFDF97FD05C0C090B102CC2058
:1018E00009F453C0D090B002D1104FC031E0309312
:1018F000B802EC01DF77209709F04AC041E040933D
:10190000B90246983FE9C32E3FE0D32EE12CF12CDB
:10191000CAEFD0E0E0911D0AF0911E0A09958111ED
:1019200003C051E05093B902E090B802EE2029F0D4
:10193000F090B902FF2009F43EC05F988BDF00975A
:10194000F1F19C01DE010E940833DC01CB0129E0AA
:10195000B595A795979587952A95D1F71092900000
:101960006AE060939100D0929900C09298008093B1
:10197000BA029093BB02A093BC02B093BD027091D7
:1019800071007260709371008FCF1092B802B1CF66
:101990009E0150E040E060E472E48FE090E00E943D
:1019A000CA3269017A0181E0C81AD108E108F10858
:1019B0001092B902AFCF4699C0CF5F9ABFCF8FEFD9
:1019C0009FEFDC01CBCFB0E0A0E0E9EEFCE00C94AF
:1019D00055334901D02EFC2DC02FD0E0DE01A80FD9
:1019E000B91F1A161B060CF06BC09B012E0D311D82
:1019F000121613060CF064C0603471050CF060C060
:101A00004115510509F45CC0062F0770702E8B013B
:101A100077FF02C0095F1F4FE3E015950795EA9530
:101A2000E1F7302F77FF04C0772011F03FEF300F40
:101A300000271127081B190B97FD02C010E000E0DA
:101A400060E8F62EF81AA038B1050CF4FD2CF01A57
:101A5000632F032E000C770BC62EC0943F3F0CF073
:101A6000C12CB1E0EE2DE77009F4B0E0E694E69405
:101A7000E694EB0E6E0D711D693071051CF028E0C7
:101A8000E22EE31AEC183C0D60E83603D001112475
:101A9000A80FB91FA00FB11FDC9C000D111D112450
:101AA000400F511FA72C072C000CBB08F33009F482
:101AB0000CC158F4F13009F4BDC0F23009F462C031
:101AC000CDB7DEB7EDE00C947133FA3F81F1232FEF
:101AD0002E0DFB3FA9F7321799F3A154BA4F8A0193
:101AE000CD018F5B9540702F741B7F1508F098C057
:101AF000F801849190E00A2C02C0880F991F0A9483
:101B0000E2F737FD05C0FC91E82FE095FE23FC933A
:101B1000772049F037303CF4FD01E058FF4F9095B5
:101B20006081692360830F5F1F4F1196D9CF232FE8
:101B30002E0D321729F2A154BA4F8A01CD018F5BC5
:101B40009540702F741B7F1508F060C0F8018491D8
:101B500090E00A2C02C0880F991F0A94E2F737FD23
:101B600003C0FC91F82BFC93772041F0373034F41C
:101B7000FD01E058FF4F6081692B60830F5F1F4FAD
:101B80001196DCCF6FEF70E0072C02C0660F771F55
:101B90000A94E2F760957095D72E732F7E0D371754
:101BA00009F48ECFA154BA4F4A01CD018F5B954005
:101BB000182D141B1F1500F5F401849190E00A2CD8
:101BC00002C0880F991F0A94E2F737FD04C01C91E8
:101BD0001623182B1C93772051F0373044F48D01D5
:101BE00000581F4FF80120812D21292B2083FFEF62
:101BF0008F1A9F0A1196D9CF3F5F4C0F5D1FA0E847
:101C0000B0E0AF19B109A80FB91FC9CF3F5F4C0FA2
:101C10005D1FA0E8B0E0AF19B109A80FB91F89CFC7
:101C20003F5F4C0F5D1FA0E8B0E0AF19B109A80FEE
:101C3000B91F51CF080D191D232F2E0D321709F48E
:101C40003FCFA154BA4F48016A01CD018F5B954047
:101C5000FC2DF41BFF1568F5F401849190E00A2C2B
:101C600002C0880F991F0A94E2F780959095F601BB
:101C7000649170E00A2C02C0660F771F0A94E2F7A5
:101C800037FD04C0EC91E823E62BEC93772049F074
:101C900037303CF4FD01E058FF4F60816923672B2A
:101CA0006083FFEF8F1A9F0A8FEFC81AD80A119628
:101CB000CCCF3F5F4C0F5D1F0C0F1D1FA0E8B0E0A5
:101CC000AF19B109A80FB91FB9CF8F2D90E0FA0154
:101CD000E00FF11FA154BA4F60E870E0681B790B68
:101CE000C81BD90B8E01000F111F41E050E06A01A3
:101CF000072C02C0CC0CDD1C0A94E2F7432F2F2DD9
:101D00003E2DCF93DF93ED01EF96EF9622968590CF
:101D1000A590772059F08C9C4001AC9C5001473035
:101D20002CF4E880B094EB20E928E992442332F0C7
:101D3000EC90A094EA20E828ED9201C011962A9533
:101D400031F73A9551F02F2D43951124E00FF11DF5
:101D5000A60FB11DC60FD11DDACFDF91CF9111248F
:101D6000AFCE90E0DECC0895282F9FB19095907F64
:101D7000669B98601C9B9460922381E0921380E0A4
:101D80000895CF93DF93EC018091CB02882389F0F3
:101D90003091D202332319F19091D902992311F194
:101DA000A091E002EBEDF2E0AA2329F0F0E0E0E000
:101DB00012C0E6ECF2E0A3EEB3E030E084E0CF3A0C
:101DC000D807B9F4BFEFB683DFEFD58371836083A3
:101DD000538342832483CF01DF91CF910895EDECAB
:101DE000F2E0E9CFE4EDF2E0E6CF3F5F189638315C
:101DF00059F3CA17DB07C9F73683E6CF8032D0F430
:101E00006831C0F490E2699FF0011124E80FF11DE0
:101E1000F595E795E05DFE4F208180FF08C02F70AB
:101E200080E1489FA0011124242B20830895207F66
:101E3000422B40830895803290F4683180F490E220
:101E4000699FB0011124680F711DFB01F595E7959D
:101E5000E05DFE4F808160FD82958F7008958DE07A
:101E60000895672F892FE7DF91E0893008F490E02B
:101E7000892F0895B0E0A0E0E0E4FFE00C9458332F
:101E8000C82EE42EFF24F394F80E0FEF060F1FEF79
:101E9000180FC1E0C60F93E0D92EBF2CBC18D0E0BC
:101EA000AD2EA10E602F8A2DC6DF8E1501F16C2F8D
:101EB0008A2DC1DF8E15D9F0AD2EA00E6A2D812F8F
:101EC000BADF8E15A1F06A2D8F2DB5DF8E1579F052
:101ED000DF5FDD11E5CF82E0D82EDD0EF3940150F7
:101EE0001150CF5F81E4D812D8CFBB24BA948B2D88
:101EF000CDB7DEB7EAE00C94743390E2699FB0018D
:101F00001124860F972F911DFC01F595E795E05D53
:101F1000FE4F908180FF04C0892F82958F700895B5
:101F2000892FFCCF88DF91E08D3008F490E0892F75
:101F300008950F931F93CF93DF93182F062FD0E0B0
:101F40006FEF600FEFDFC0E0882311F0D1E0C1E058
:101F5000602F81E0810FE6DF882311F0D260CF5F30
:101F600061E0600F812FDEDF882311F0D460CF5F46
:101F7000602F8FEF810FD6DF882311F0D860CF5FFD
:101F80008D2F9C2FDF91CF911F910F910895B0E07D
:101F9000A0E0EDECFFE00C9450337C016B018A0172
:101FA000E90197FF02C081509F4F892E992E990C0D
:101FB0009908C80117FF02C081509F4F292E392E62
:101FC000330C33088214930409F45EC08214930422
:101FD0000CF0CFC054018FEFA81AB80ABA2CAA246B
:101FE000AE18BF0844244394512CBE016C197D09DE
:101FF000072E000C880B990B982F872F762F6627BA
:1020000098012E193F0937FF03C0319521953109F9
:10201000032E000C440B550B0E94CA3266246A94AE
:102020007FE7772E211580E838074105510554F4E4
:102030003901213030484F4F5F4F24F466246394B8
:1020400060E8762E9301D5010E94443320E031E010
:1020500040E050E00E94CA325601A20EB31E840C2A
:10206000951C240C351CC501B7FE02C081509F4F42
:10207000A60CB71C692F882D55DF81118EC0840CEA
:10208000951C2814390479F7C601D7FE02C0815087
:102090009F4FA92EB92EBB0CBB08CE01D7FF02C0A3
:1020A00081509F4F492E592E550C5508A414B50444
:1020B00009F459C0A414B5040CF065C035018FEFC4
:1020C000681A780A762C66246C187D088824839414
:1020D000912CB8016E197F09072E000C880B990B03
:1020E000982F872F762F66279E012C193D0937FFE1
:1020F00003C0319521953109032E000C440B550B7B
:102100000E94CA32CFEFDFE7211580E8380741058A
:10211000510544F4E901213030484F4F5F4F14F42A
:10212000C1E0D0E89E01D3010E94443320E031E0B9
:1021300040E050E00E94CA32E20EF31EA80CB91C27
:10214000480C591CC701F7FE02C081509F4FEC0E8E
:10215000FD1E6A2D892FE6DE81111FC0A80CB91C57
:102160004A145B0479F781E0CDB7DEB7E2E10C9465
:102170006C33C70160E071E00E942B335C014424A2
:102180004A94542C32CFC60160E071E00E942B3398
:102190003C0188248A94982C9CCF80E0E5CF9091D4
:1021A000BC03981731F08093BC031092BB031092CC
:1021B000BA030895CF93DF93EC01605284E0689FE7
:1021C000B001112463567C4FFB01249124272883FE
:1021D0003196E491E427E983FB0132963491342768
:1021E0003A83FB013396549154275B83DF91CF915F
:1021F0000895A5E0B0E0EFEFF0E10C945A3320E849
:10220000629FB0011124460F572F511DFA01E1546E
:10221000FA4F7F01009721F19E012F5F3F4F690127
:10222000F90110E000E00F5F1F4F6AE070E00E94CC
:102230001733805D8193CB010530110511F00097B4
:1022400091F70C0D1D1D0C151D0571F04FEFD801F8
:102250006E918D01C701AEDFF4E0EF0EF11CF3CFFC
:102260004FEF60E3CF01A6DF2596E8E00C947633CC
:10227000EF92FF921F93CF93DF93122F119520E8D7
:10228000629FE0011124C40FD11DC154DA4F7C01BB
:10229000F7016491FFEFEF1AFF0A662329F0412F3F
:1022A000CE0188DF2496F4CFDF91CF911F91FF906C
:1022B000EF90089580910001909101019C01369565
:1022C000322F22273795279528273927C901892FAB
:1022D0009927869528273927922F882782279327A1
:1022E00090930101809300010895EF92FF920F9364
:1022F0001F93CF93DF93FC012091E602822F8E7F04
:10230000C2EED2E0C9F030910B03032F0E7FC7E07D
:10231000D3E091F090913003192F1E7FB1F13695E3
:102320002695C7E0D3E0321710F0C2EED2E09695C2
:10233000EC80E6949E1548F1F983E8837B836A83F9
:10234000FC8040FBF0F8FC827E0185E2E80EF11C87
:102350008E010B5F1F4FE016F106D1F0ABDF8F71DE
:102360008051D8018C93A6DF8F718051F801818351
:10237000A1DF8F718051F80182839CDF8F718951B9
:10238000F80183830C5F1F4FE6CFCCE2D3E0D4CFBC
:102390004C8141704C624C83CDB7DEB7E6E00C94C3
:1023A0007833ACE0B0E0E7EDF1E10C945033982ED7
:1023B0006C87842E722E102FE982112339F0298127
:1023C000222321F040E0622F812F18DD38E03815FC
:1023D00008F43FC1371508F440C11B8641E01C8555
:1023E000123008F440E09B8540FB94F99B8751E054
:1023F000591508F050E02B8450FB27F82B86E92C68
:10240000F12C882D90E09E838D836C01CE0CDF1C17
:1024100071E09EE1C916D1040CF070E03B8470FBC2
:1024200035F83B860C8510E0872D90E098878F83E8
:102430005C01A00EB11EA1E096E1A916B1040CF05A
:10244000A0E04B84A0FB46F84B866C856250698304
:1024500044244A94490C842D50DD682C690C88234F
:1024600041F06981862D49DD882319F0BB85BF7E47
:10247000BB873C843A948EEF890D8A83632D3DDDC2
:102480005C84570C882341F0652D8A8136DD8823D2
:1024900019F0EB85EF77EB8781E0860D8C83632D58
:1024A0002CDD882351F06C856F5F670D862D25DD4F
:1024B000882319F0FB85FF7DFB8761E0650D6B8349
:1024C000842D1BDD882341F06B81862D16DD88234A
:1024D00019F02B852F7B2B876981842D0EDD8111CF
:1024E00009C0632D8A8109DD811104C03B853F7ECF
:1024F0003F773B876981862D00DD811109C0632DFF
:102500008C81FBDC811104C04B854F7E4F7D4B8756
:102510006B81862DF2DC811109C0652D8C81EDDC8B
:10252000811104C09B859F7B9F7D9B876B81842D40
:10253000E4DC811109C0652D8A81DFDC811104C0D2
:102540005B855F7B5F775B87632D892DD6DC882376
:1025500041F0632D8FEF860DD0DC2224239481116E
:1025600001C0212C6C85862DC8DC882341F06FEFDB
:10257000650D862DC2DC71E07987811101C0198655
:10258000652D892DBADC882341F0652D8FEF860DEE
:10259000B4DCA1E0AA87811101C01A866C85842D64
:1025A000ACDC882339F06FEF650D842DA6DCB1E03B
:1025B000811101C0B0E0211005C0EB85EF7EEF7DF9
:1025C000EF77EB878985811105C0FB85FF7EFF7D55
:1025D000FF7BFB876A85611105C02B852F7D2F7BD3
:1025E0002F772B87B11105C03B853F7E3F7B3F771F
:1025F0003B87EC14FD040CF0E7C02E2C632D8E2DD0
:102600007CDC811103C04B8541604B87652D822D99
:1026100074DC811103C09B8594609B875C8552307C
:1026200040F06981822D69DC882319F07B857F7EEB
:102630007B8796E1A916B10444F46B81822D5DDCA1
:10264000882319F0AB85AF7BAB873FEFE31AF30A22
:10265000D0CF0FEF871408F05CC01FEF2BDE272DC3
:102660002650330BB9010E94173323E0F22EF80EE7
:10267000EE24EA94E90C115009F4AFCE6C856F0D8D
:1026800069838E2D3ADC882349F3082D090D698171
:10269000802F33DC882311F3D980DA946D2D8E2DB1
:1026A0002CDC8823D9F26D2D802F27DC8823B1F212
:1026B000B980B3946B2D8E2D20DC882379F26B2D9D
:1026C000802F1BDC882351F2F5DDC82CD12CB601FC
:1026D000625071090E94173311E0190D180F092D6E
:1026E000C601890D911D0817190634F44DE0698162
:1026F000802F84DB0F5FF4CF2FEF270D2F19E98098
:10270000012F482D6B2D892D4CDE7F2CF82C8F2C22
:1027100054CED0DD282D2650330BB9010E9417333B
:1027200093E0F92EF80EEC84EA94015009F455CEAA
:102730001F2D190D6E2D812FE0DB882351F36C8541
:10274000670D6983812FD9DB882319F355245A94A7
:10275000510E6E2D852DD1DB8823D9F26981852D0F
:10276000CCDB8823B1F266246394610E6E2D862D36
:10277000C4DB882371F26981862DBFDB882349F28F
:1027800099DDC72CD12CB601625071090E94173314
:102790000C850F5F080F09830C855601EC84AE0C85
:1027A000B11C0A151B0434F44DE0602F812F26DB89
:1027B0000F5FF3CF4FEF480D4F19E980012F272D01
:1027C0006C85862DEEDDA3CF0A151B055CF5F02E7A
:1027D000602F842D92DB811103C0BB85B860BB875D
:1027E0006F2D862D8ADB811103C0EB85E260EB87BC
:1027F00081E0891540F46F2D8A817FDB882319F0F1
:10280000FB85FF77FB878EE1C816D10444F46F2D5A
:102810008C8173DB882319F06B856F7D6B870F5F6D
:102820001F4FD2CF2B8525FB112710F926FB002740
:1028300000F927FBFF24F0F824FF07C03BDD64E626
:1028400070E00E941733449760F1FF2039F032DDC9
:1028500064E670E00E941733449790F1002339F04A
:1028600029DD64E670E00E9417334497C0F111231C
:1028700009F444C01FDD64E670E00E9417334497FA
:1028800008F03CC010E000E04F81588504171507A0
:10289000ACF56C85600F40E0862DB0DA0F5F1F4FFE
:1028A000F3CF10E000E08D819E810817190734F501
:1028B00040E0632D892D800FA1DA0F5F1F4FF3CF0A
:1028C00010E000E0EF81F8850E171F07BCF46C855F
:1028D000600F40E0842D92DA0F5F1F4FF3CF10E0BE
:1028E00000E0AD81BE810A171B0744F440E0652D6E
:1028F000892D800F83DA0F5F1F4FF3CF87101AC027
:1029000036E03815B8F46C856F5F698393944DE0B9
:10291000892D74DA6A946A944DE06981862D6EDAA5
:102920005A945A944DE0652D862D68DA4DE0652D58
:10293000892D64DA2C96E2E10C946C33FC01408121
:102940005181DB012D913C91F901E05CF1094E17B9
:102950005F07BCF020543F4F2417350794F0FC016B
:1029600042815381FB0122813381B901605C71098D
:102970004617570734F060587E4F81E0641775079B
:102980000CF480E00895262FFC0142815381608180
:102990007181F7D921E0892B09F420E0822F089575
:1029A000FC012091AF043091B00480819181281BFB
:1029B000390B37FF03C0319521953109932F2091B1
:1029C000B1043091B20442815381241B350B37FF8F
:1029D00003C0319521953109892F931708F4832F6E
:1029E00008950F931F93CF93DF93EC01062F142FBD
:1029F000642F802F20DA893080F5612F8E811BDAD9
:102A0000893058F56F81802F16DA893030F5E3EE82
:102A1000F3E0EC17FD07A1F084818770843081F02A
:102A20002681402F002E000C550B2417150641F46B
:102A30003781612F012E000C770B3617170669F0CE
:102A4000389684E0E33AF80721F70E831F8381E08C
:102A5000DF91CF911F910F91089580E0F9CFFC0194
:102A600084818770843039F0FAE08F9FC00111248F
:102A70008B589C4F089590E080E00895CF93DF93AA
:102A8000C3EED3E09C819770943089F46883798396
:102A90004A835B8387708C837E835F83CE01DFDF15
:102AA0000296FC0184918D83DF91CF910895289641
:102AB000F4E0C33ADF0731F7F7CF2091A503E1E552
:102AC000F3E050E040E0942F421798F19091A50375
:102AD0009C3008F47CC0292F2150330BB90127E02A
:102AE000269FF001279FF00D1124EF5AFC4F2681FD
:102AF000281708F04BC040E0242F30E02617370796
:102B00000CF06AC087E0829FD001839FB00D112432
:102B1000AF5ABC4F2F5F3F4F829FF001839FF00D54
:102B20001124EF5AFC4F01900D928A95E1F74F5F07
:102B3000E3CFBA0136814F5F5F4F3796831718F6A0
:102B40002C3008F551E0520F5093A50377E0279FF2
:102B5000D0011124AF5ABC4FBD0167507109FB0170
:102B600037E001900D923A95E1F72150DB01921781
:102B700098F39C3009F4AACFF7E09F9FC00111247D
:102B80008F5A9C4F089540E0911103C090E080E07F
:102B90000895242F30E0DB0111972A173B07E4F456
:102BA00087E0829FD001839FB00D1124AF5ABC4FA4
:102BB0002F5F3F4F829FF001839FF00D1124EF5A4A
:102BC000FC4F01900D928A95E1F74F5FE2CFB1E0A3
:102BD000B90FB093A503D0CF9150CECFA7E1B0E00D
:102BE000E4EFF5E10C9450334C01522F550F8E2D2C
:102BF00090E09A8789872150330B02C0359527953D
:102C0000EA94E2F7229FC001239F900D900D1124BA
:102C10009C012C5A3D4F3E872D87862F880F880BAD
:102C2000162F11951823852F90E09C01260F311D3A
:102C300067FD3A95213831050CF4D9C070E8761B50
:102C40007F8B242F2195442E440C44082421298B6A
:102C5000840F911D47FD9A958134910514F050E43D
:102C6000541B6E8367FD1E82D12C662777276C1953
:102C70007D09788B6F8747FD40E030E1430290018A
:102C80001124C901807893709B8B8A8BB12E188692
:102C90001F82D12C30E020E0F12CE12C312C212CB2
:102CA000712C612CAE81A11BAB0D9F89B91608F068
:102CB00001C10A2E000CBB0BFD01E15CFA4F8081C3
:102CC00071E07B87801708F01B86801708F0EAC048
:102CD000EF81F885E10FF11D6F896250770BE617E0
:102CE000F7070CF486C0DD2009F4E4C0C3018E218F
:102CF0009F219C838B83D12CC12C512C412C642F80
:102D000067706A887B88A60DB71DA154BA4F9C9145
:102D1000E62FF0E0E45BFD4F8491E988F12CFD8A19
:102D2000EC8A1C861A82F0E01982A12C7C88751628
:102D300008F0B3C0A110AF2EE52FE250FF0B7F01CA
:102D4000EC89FD89EE15FF050CF093C0098402C0E3
:102D5000F595E7950A94E2F7ED84FE84EE0DFF1DEC
:102D6000E491F0E0EE0FFF1FE45DFD4FE590F4907D
:102D7000EB81FC81EE21FF2171E07D83EF2B09F4D3
:102D80001D8266246394F101EE21FF21EF2B09F4EB
:102D9000612CE222F322F1E0FE8BEF2809F41E8A77
:102DA000F980FF2009F469C0EA80EE2009F471C0BF
:102DB000982B6F5F880F683069F49C9361E0640F13
:102DC0008989681B670D603414F4A058BF4F9C912B
:102DD00081E060E0EC89FD893196FD8BEC8B7D8094
:102DE0007C86FA81FE88FA82A98069829FCF5F8BF8
:102DF00028CF098402C0F595E7950A94E2F74D843F
:102E00005E84E40DF51D849190E0880F991F880F72
:102E1000991FF401E80FF91FDD20B9F04590549097
:102E2000FC013296E80DF91DC590D4908F859889E4
:102E3000C826D926C2018C219D21E620F720B701A2
:102E4000682B792B7C836B835ACF25903490FC01BF
:102E50003296E80DF91D259134918F8598892827A0
:102E600039277101E222F322FC82EB826901210100
:102E700046CF1D821E8A612C93CFEC85E11109C0DB
:102E8000A11007C0662009F494CFAE88AA2009F4E7
:102E900090CF782F709597238CCF9C9379019601D2
:102EA00031011201B394AF81B8851196B887AF8311
:102EB000DB84F8CE6796E2E10C946C33B0E0A0E0DE
:102EC000E4E6F7E10C9454338901E8EAF3E0208169
:102ED00031817C01E21AF30A828193813B01681AF5
:102EE000790AC581D681C780D0849E01D7010E940E
:102EF0004433872E982EA92EBB24A7FCBA949601A2
:102F0000D3010E944433672F782F892F992787FD9B
:102F10009A95861A970AD8018D929C92D7010E94A1
:102F20004433C72ED82EE92EFF24E7FCFA949E01E5
:102F3000D3010E944433672F782F892F992787FD6B
:102F40009A95C60ED71EFA01D182C082CDB7DEB7E0
:102F5000EEE00C947033A4E0B0E0E1EBF7E10C9408
:102F60005A337A0169019E012D5F3F4FAE014F5FD9
:102F70005F4FA4DF0B811C81003211056CF0A98129
:102F8000BA81B7FF0BC044275527401B510B440F94
:102F9000551FA417B50754F480E025C0109731F0F1
:102FA000C801880F991F8A179B07B4F321E430E00A
:102FB0000E944A339801012E000C440B550B0E94CD
:102FC000CA32F7013183208380E890E2B8010E9481
:102FD0002B33D6016D937C9320813181205C3F4F50
:102FE0003183208381E02496E8E00C947633A4E0DA
:102FF000B0E0EDEFF7E10C9458335C01CB01BA017E
:10300000122F9E012D5F3F4FAE014F5F5F4FA3DF39
:10301000882309F446C08B819C81189F6001199F09
:10302000D00C1124D7FE03C02FE7C20ED11CCC0C4C
:10303000CD2CCC1CDD08F9802F2D3A8120383105AC
:1030400014F02FE730E037FF02C030E020E02154D9
:103050003B4FF9011081013069F138F1033061F122
:10306000FC184F2D0F2C000C550BB60177277195CE
:1030700061957109660F771F4617570794F001E0B5
:10308000080F802F1ADDFC01892B59F08281B18253
:10309000A082F3821483C58206838E7FE0FA81F9D1
:1030A00082832496EAE00C947433180F2C2D220F9F
:1030B000121BD6CF1C19D4CF181BD2CFE0E4F0E0FE
:1030C000E81BF109FF27EE0FFF1FE15EFF4E859120
:1030D0009491089587FD17C06034A8F470E090E1E2
:1030E00021E061FD24E060FD220F62FD2295687FF2
:1030F000969FD0011124A80FA154BA4F0C90022A18
:1031000040FF02260C920895A0E2B0E0EAE8F8E160
:103110000C9450335A0149010F8BEE8EC98E9E01DB
:103120002B5F3F4FAE01495F5F4FC8DE9E012F5FAF
:103130003F4FAE014D5F5F4FB401C501BFDE2B8134
:103140003C8137FF0BC089819A81919581959109C6
:10315000880F991F281739070CF4CBC3EF81F88526
:103160008D809E801E161F063CF4A401440F551F3F
:103170004E175F070CF4BDC369817A8140E2841663
:1031800091040CF0EEC0603271050CF4B2C300E2A1
:1031900010E07801E818F9081B0128183908C70160
:1031A0009695982F882797958795B1010E942B3384
:1031B00069872E1B3F0B2E9DC0012F9D900D3E9DBC
:1031C000900D1124B1010E942B33E60FF71FF887F1
:1031D000EF831E830D8310E81C871F8ACD80DE805D
:1031E000AF81B88521E430E00E944A3396010D2C6E
:1031F000000C440B550B0E94CA3249015A01098147
:103200001A81190180E4280E311CAB81BC8121E4B4
:1032100030E00E944A339801012E000C440B550BFC
:103220000E94CA3279019FE3E90EF11C2E143F047B
:103230000CF05FC31E141F040CF05BC3E0E82E16F5
:1032400031040CF056C320E830E2C901B6010E94F7
:103250002B333B01C901B8010E942B337C8B6B8B54
:1032600037FE2AC000EC1FEF081919094701821820
:103270009308092C000CAA08BB086C858985681B7B
:10328000770B9B01D8010E944433A50194010E9451
:10329000CA329985920F99872B893C89261937095B
:1032A000D8010E944433A50194010E94CA32620EE3
:1032B000731E1F8A312C212C6701C218D308DA8AA9
:1032C000C98A2601D7FE03C0FFEF4F1A5F0A559443
:1032D0004794AB89BC896A167B060CF071C0A619AD
:1032E000B709BD8FAC8F31E03A872B8EFE8AED8A0D
:1032F000E0E8EE16F10424F04FE750E05E8B4D8BD2
:10330000DD88DF8E63018101D801A154BB4FBC91E0
:10331000BD8717FD08C0F801E15CFA4FF081FC158C
:103320001D040CF4E1C2798D772309F40FC150E03C
:10333000C801809590958170552309F407C1BF8815
:10334000BB2021F02016310609F444C0AE8CAA201F
:1033500019F0E016F106F1F14FEF8823E1F145E5B0
:103360003AC06032710544F500E210E05801A61A37
:10337000B70A861A970A50E8B5015603C001579F4D
:10338000900D1124B4010E942B3360586C87E21B0E
:10339000F30BEA9DC001EB9D900DFA9D900D112459
:1033A000B4010E942B33260F371F3C832B831A83D3
:1033B000098319861E8E12CF70E87C8719860ECF7E
:1033C000F3018B899C89E81BF90BFD8FEC8F9FEF34
:1033D0009A878BCF40E08C2D91E4C916D1040CF074
:1033E00080E46D85680FBD84B81AA02E6B150CF4AF
:1033F0003AC067FD38C09FE39B15ACF1EB2DB7FCDD
:10340000E0E0862F60340CF08FE3980133272154DD
:103410003A4FA0E1EA9FD0011124A078B370A20F27
:10342000B31F70E1879F4001112490E8892293E047
:103430009922280D391DE770F0E0E959FC4E87709C
:1034400090E0815A9C4EA217B30709F061C0249105
:10345000FC01E4917E2F7223F72FF0959C91F923C4
:1034600074237F2B7C9340E08A2D34DE40E06B2D6B
:103470008A2D30DED801A15CBA4F6C91611105C074
:103480004091BE044F5F4093BE042FEFC216D1049B
:1034900009F00CF457C08FEF8C93B1E0BF87E016B2
:1034A000F10609F461C08C8C9D8C481859089A84E7
:1034B000892C990C9908C4018C0D9D1D88A3BD848D
:1034C000B81AB88A560157FEC0C0A80CB91C298981
:1034D0003A89420E531E3F853323A9F057FE13C08D
:1034E00081E2A816B1047CF46A856095E8A16E0FAC
:1034F0006C197D85670F6A0D40E0802FEBDD40E0A1
:103500006889802FE7DDF8899A85F91BF88BDBCF76
:10351000E491FE2FF0955C91F523E423EF2BEC93DF
:10352000A058BF4F2A173B0711F04C93F9CFFC016D
:10353000B4918B2F8095F901308183234B23482B45
:10354000408391CFCC9251E05F87A9CF6B8D6017FC
:10355000110621F46F5F6B8F1F86A1CF2D893E89E5
:1035600002171307CCF70F8FAB8D6F8DA61709F4D9
:10357000C0C134E0631671040CF4BBC14B895C8993
:10358000443051050CF4B5C15C858985581709F4A0
:10359000B0C1BFE64B2EB3E15B2EF201F491FF8781
:1035A000BF85BB2309F4A5C1B150BF87F201319695
:1035B0004491319614913196249134E0430E511C7C
:1035C000F2019490F9852F1758F33C85341740F396
:1035D000A92CB12CCF2ED12CE32EF12C4F17C0F4F7
:1035E0004217D9F150E0D601A41BB50BB501611B00
:1035F0007109A69FC001A79F900DB69F900D112441
:10360000622F70E0641B750B0E942B33160F4F2F37
:103610000C85021718F52417B1F030E0F701E21B12
:10362000F30B612F70E06A197B09E69FC001E79FE9
:10363000900DF69F900D1124642F70E0621B730BA8
:103640000E942B33960E2C8509C00F5F1F4F003848
:1036500011050CF089CF650157CE4985EC18FD089E
:10366000842F90E08C199D099695982F882797951F
:103670008795B7010E942B33062F30E02C193D09A6
:10368000C9019695982F882797958795B7010E942D
:103690002B33E62F202F30E0A989BA890E944A33C4
:1036A000F7E09595879577956795FA95D1F751014C
:1036B000A60EB71E2E2F30E00E944A336B017C010C
:1036C000A7E0F594E794D794C794AA95D1F7C20CD4
:1036D000D31CCA14DB040CF463CFEB88FC88E61817
:1036E000F7080E9DC0010F9D900D1124880F892FA2
:1036F000881F990B860D971DEE9D9001EF9D300D53
:103700001124220F232F221F330B260D371D929ECB
:103710007001939EF00C112456E0F594E7945A95AD
:10372000E1F740E250E0DA01A21BB30BEA0EFB1E08
:10373000189FF001199FF00D11248F0166E0159577
:1037400007956A95E1F7481B590B040F151F17FFE2
:103750009FC0F7FC25CF45018C189D08809EC001B5
:10376000819E900D909E900D1124B701601B710BEE
:103770000E942B33A60EB71E10E000E0F0E4EF1617
:10378000F1040CF08EC08B8C912CA814B9040CF0B1
:10379000A1C0CA14DB04A1F0D401AA19BB09B70166
:1037A000601B710BA69FC001A79F900DB69F900D47
:1037B0001124B6016A197B090E942B33060F171FCB
:1037C000C601881999099E878D875C0197FF03C000
:1037D0007FEFA71AB70AB594A7940E151F050CF032
:1037E0007BC09701201B310B388F2F8B91E0988B7A
:1037F000A40141545B4F5A8F498FC814D9040CF46B
:10380000CFCE5F8D581519040CF4CACEA98DBA8D90
:10381000FD91BA8FA98FFD8B0C8F8E8E60EE600F9D
:103820006F0F40E0882D56DC6F89788DA61AB70A95
:103830001B870A87B7FE26C0B8898B2F0B2E000C7A
:10384000990BEA85FB85E80FF91FFB87EA872D8531
:103850003E85A20EB31EB7FE0DC0800F911F682FCC
:103860006B1B60523C8D631B8D89680F6E0F40E0AF
:103870008E8D30DCC814D904E9F6EA85FB85EE1696
:10388000FF06C1F67FEF871A970A0A851B85B5CF19
:1038900020E4E216F1040CF476CF003411050CF0AC
:1038A0007FCE2FE330E02E193F09A5014C195D09A9
:1038B000249FC001259F900D349F900D1124B801C5
:1038C0006E197F090E942B33C60ED71E9FE3E92E87
:1038D000F12C59CF450174CFF801EE19FF09F88F8B
:1038E000EF8B7FEF788B84CF898D598D811120CD1F
:1038F00026CDA096E2E10C946C33B0E0A0E0E3E8C2
:10390000FCE10C945333E82EF62E0E941B0FCF2DB2
:10391000D0E00E2D10E06091B1037091B203909150
:10392000B503D801A91BB109E091B303F091B40329
:10393000A090B603AE014A1951096A9F90016B9F8E
:10394000300D7A9F300D1124E49F5001E59FB00C9B
:10395000F49FB00C11242A193B0921153E4F0CF499
:1039600049C0AE9F9001AF9F300DBE9F300D112416
:10397000649FD001659FB00D749FB00D11242A0F74
:103980003B1F21153E4F0CF435C082508B3008F0A0
:10399000EDC0E82FF0E0E153F34E0C943E33DA1C17
:1039A0002A1D381D541D701D7E1D621D461D9A1D49
:1039B000A81D8C1D8091A703EAE6AE2EE8E0BE2E7E
:1039C00082FF04C07AEAA72E78E0B72E6F2D8FEF22
:1039D0008E0D0E94920F882391F05C2F442740584F
:1039E0005F4F702F66276C5D7F4FE12C01E02BE469
:1039F000C501FDDACDB7DEB7EFE00C946F336F2D64
:103A000081E08E0D0E94920F882349F05C2F44279D
:103A100040585F4F702F662765527F4FE6CF6FEF9C
:103A20006F0D8E2D0E94920F5C2F44274C5D5F4FCF
:103A300081110BC061E06F0D8E2D0E94920F8823C3
:103A4000C9F25C2F442745525F4F702F662760589C
:103A50007F4FCBCF5C2F442740585F4F702F662796
:103A600060587F4FE12C03E020E68CEE91E0C1CF5F
:103A70005C2F442740585F4F702F662760587F4F58
:103A8000E12C00E020E68CEA91E0B3CF5C2F4427E4
:103A900040585F4F702F662760587F4FE12C00E041
:103AA00020E58CE691E0A5CF5C2F442740585F4F7E
:103AB000702F662760587F4FE12C00E020E48CE2F5
:103AC00091E097CF5C2F442740585F4F702F6627B7
:103AD00060587F4FE12C00E020E480EE9DE089CF2C
:103AE0005C2F442740585F4F702F662760587F4FE8
:103AF000E12C00E020E480EA9DE07BCF5C2F4427AE
:103B000040585F4F702F662760587F4FE12C00E0D0
:103B100020E480E29EE06DCF5C2F442740585F4F49
:103B2000702F662760587F4FE12C00E020E58CEE77
:103B300090E05FCF5C2F442740585F4F702F66277F
:103B400060587F4FE12C00E02BE480E69EE051CFEF
:103B50005C2F442740585F4F702F662760587F4F77
:103B6000E12C00E02BE48CEA90E043CF3091BE04DE
:103B700037FD40CF6F2D8E2D0E94920F882309F4C0
:103B800039CFB02EAA24DC2FCC27450193943E01D7
:103B900073946F2D8FEF8E0D0E94920F582E6F2D04
:103BA00081E08E0D0E94920FD82E6FEF6F0D8E2D3B
:103BB0000E94920F182F61E06F0D8E2D0E94920FC0
:103BC000F82E511025C06091A8037091A9036A15C1
:103BD0007B05F4F4811109C0EE24E394E091AA037B
:103BE000F091AB03E615F7050CF0E12C111108C0BC
:103BF00001E04091AA035091AB03C417D5070CF024
:103C000000E0CC24C3949301A501BE01C5017CDA78
:103C1000F11024C02091AA033091AB036216730601
:103C2000ECF4D11009C0EE24E394A091A803B09164
:103C3000A903A815B9050CF0E12C511008C001E04A
:103C40008091A8039091A903A816B9060CF000E092
:103C5000C12C9301A401B301C50156DAD11025C0CE
:103C60006091A8037091A90386169706F4F41111C8
:103C700009C0EE24E394E091AA03F091AB03CE17C0
:103C8000DF070CF0E12CF11008C001E04091AA031D
:103C90005091AB03461557050CF000E0CC24C394BB
:103CA0009E01A401B301C4012FDA1111A3CE20910A
:103CB000AA033091AB032C173D070CF09BCE51109B
:103CC00009C0EE24E394A091A803B091A903AA1619
:103CD000BB060CF0E12CD11009C011E08091A803C3
:103CE0009091A903881599050CF010E0C12C012FC3
:103CF0009E01A501BE01C40107DA7CCECF92EF92EE
:103D0000FF920F93CF93DF93213490F4CE2CD42FD6
:103D1000C62F32E0E32E213238F4422F50E04131F9
:103D200051056CF0EE24E3944D2F6C2F0E94EE159C
:103D3000DF91CF910F91FF90EF90CF900895E12CFC
:103D4000233090F7462F660F550BBA01615C7A4F0E
:103D50007B01FB0180812230D1F4801748F440E0E0
:103D60006D2F8C2FB7D940E061E06D0F8C2FB2D949
:103D7000F701C180C016E0F6CF5F40E06D2F8C2FB9
:103D8000A9D961E06D0F40E08C2FA4D9D1CF801765
:103D900078F640E06D2FF8CF9C01E1E7F0E09081EC
:103DA0009D7F908381E08093B7023093B602209389
:103DB000B5023093B3022093B2020C943E0C0895E6
:103DC000CF93C82F8091B904863018F426E0209351
:103DD000B90438E03093BA044091BC04C41738F0F9
:103DE00089EC92E1D9DF1092BC04CF9108958FE164
:103DF00092E1D2DF5091BC045C1B5093BC04F5CF20
:103E0000B0E0A0E0E6E0FFE10C945833C091AF04CD
:103E1000D091B0048091B30451D92CE3AC01249F1C
:103E2000C001259F900D112497FF02C081509F4F24
:103E3000A92EBB24A7FCBA94CA0DDB1DE091B304E4
:103E4000F0E0EE0FFF1FE15EFF4EC590D4903CE323
:103E50003C9D80013D9D100D112417FF02C00150B3
:103E60001F4FA12EBB24A7FCBA94E090B104F090A0
:103E7000B204AE0CBF1CCE01D7FF02C081509F4FD1
:103E8000D92E7501B7FE03C05FEFE50EF11C6F2D53
:103E90008D2D0E941B0F8A3009F451C08C3009F41B
:103EA0006AC00091B1041091B204580180E3A81ACD
:103EB000B108E090AF04F090B0046701E0E3CE1ADF
:103EC000D108B501C6010E94310FD82F811131C030
:103ED000F0E3EF0EF11CB501C7010E94310FD82F9E
:103EE000811127C0005D1F4FB801C7010E94310F2B
:103EF000D82F81111EC0B801C6010E94310FD82FE2
:103F0000811117C003EE13E083EAE82E84E0F82E57
:103F1000F80194819770943039F06FEA74E0C80129
:103F20000E949E14811131C0085F1F4FE016F106F8
:103F300079F78D2FCDB7DEB7EAE00C9474334BE000
:103F40006F2D8D2D0E94FE0E41E0B501CE010E9425
:103F5000751181EE9FE020DFA1ECBFE0B093A504D6
:103F6000A093A4045AE55093A3047091AB047F5F1F
:103F70007093AB0496CF62EA7FE07093A5046093E0
:103F8000A4041AE51093A3048CCFD82FD2CFCF93DB
:103F900088E00E94B40EC0E1811101C0C0E084E05D
:103FA0000E94B40E8111C06280E80E94B40E81119B
:103FB000C46080E10E94B40E8111C86080E20E945A
:103FC000B40E8111C16080E40E94B40E8111C26000
:103FD0008C2FCF9108951F920F920FB60F9211243C
:103FE0008F939F938091E1009091E100937F909354
:103FF000E10083FF0FC01092E90091E09093EB0085
:104000001092EC0092E39093ED001092E20398E09E
:104010009093F00082FF22C093E09093E90090918A
:10402000F200992319F09AE39093E8009091D3035A
:10403000992341F09091D30391509093D303911120
:1040400001C05D9A9091E103992341F09091E103C1
:1040500091509093E103911101C0289A84FF18C0F8
:104060009091E2009E7E91609093E2008091E10049
:104070008F7E8093E1008091D4038E7E8061809357
:10408000D4039F918F910F900FBE0F901F901895A2
:1040900080FFF7CF8091E2008E7E80618093E20006
:1040A0009091E1009E7E9093E1008091D4038E7EFA
:1040B0008160E5CF1F920F920FB60F921124CF921D
:1040C000DF92EF92FF920F931F932F933F934F93A3
:1040D0005F936F937F938F939F93AF93BF93EF9370
:1040E000FF93CF93DF93CDB7DEB76C97DEBFCDBF25
:1040F0001092E9008091E80083FF25C068E0CE01BE
:1041000045960E94840B02EF0093E8001D8917FF7B
:1041100039C0C090E800C0FEFCCF212F207609F006
:1041200033C13E894F89588D6F89F88C311131C068
:10413000103861F5F090D203F092F1001092F10086
:10414000FEEFF093E8006C960FB6F894DEBF0FBE5A
:10415000CDBFDF91CF91FF91EF91BF91AF919F9133
:104160008F917F916F915F914F913F912F911F910F
:104170000F91FF90EF90DF90CF900F900FBE0F90B8
:104180001F9018959EEF9093E800C7CF1092F10012
:10419000D5CF313059F41111D3CF4130510581F6CB
:1041A0008091D2038D7F8093D203CACF333049F4FC
:1041B0001111C6CF4130510519F68091D2038260AA
:1041C000F2CF353041F4D090E800D0FEFCCF6068EB
:1041D0006093E300B5CF363009F0A8C00B8D1C8D7D
:1041E00092E01092E9001092D0031092CF03F912DE
:1041F0002EC01092CE031092CD030E94590B1F8245
:1042000059E05983FA8271E07E83B0EAB8872AEFD9
:1042100029874091CF035091D003475F5F4F5C8364
:104220004B838D831092E9001092D0031092CF033C
:104230001093CE030093CD0349E050E0BE016F5FC1
:104240007F4F80E00E94380B0E94590B79CF10936A
:10425000CE030093CD030E946F0AFC01C280D3807D
:10426000C114D10409F452C1D601ED91FC9104802E
:10427000F581E02DBE016B5E7F4FC6010995009769
:1042800009F03FC1F601C084D184EACF33E0F312D4
:104290000EC04F89442309F440C0423061F440E825
:1042A00067E08AE99FE00E940B0B811149CF61E230
:1042B0006093EB0048CF413029F440E86BE08EE892
:1042C0009FE0F1CF433099F70E946F0AFC01C28052
:1042D000D3808E010F5F1F4F7801C114D10479F094
:1042E000D601ED91FC910680F781E02DB801C60161
:1042F0000995080F111DF601C084D184EECFD801B5
:104300001C92F70101900020E9F7BF01615071098B
:104310006E197F0940E0C701C6CF68E77FE0FB0167
:10432000449150E080E80E94380B0ACF373009F4FE
:10433000BECF383021F4F1E0F093F10001CF3930F5
:1043400009F0FECE137009F0B2CFE1E1F1E081E0B7
:104350005191552381F08093E90071E07093EB0057
:10436000DF011197CC90C092EC00B6E3B093ED0062
:104370008F5F873069F72EE72093EA001092EA00FA
:10438000EF88E092E203DCCEEB8CFC8C1092E9002B
:104390001092D0031092CF03F092CE03E092CD039F
:1043A000D98CD11094C03E894D89413A49F43132BB
:1043B00009F07DCF47E050E068E071E080E0B3CFE6
:1043C000413209F074CF333269F48F89988DB0E0AF
:1043D000A0E08093040190930501A0930601B0939F
:1043E0000701AECE303269F4D090E800D2FEFCCFA7
:1043F00067E088E091E00E94840B0BEF0093E800F7
:104400009FCE323209F09CCEFF88F0920F01EEEF82
:10441000FFE7659174916B3F7C4D51F1E0E0F8E06E
:104420008091080190910901A0910A01B0910B01BE
:10443000803B9440A105B105F1F450910F0150FD6E
:104440001AC0EE3F8AE0F80791F5A7E7B7E7B18316
:10445000A083F0916000F093D10318E19BE00FB6C8
:10446000F894A895109360000FBE9093600068CEFA
:10447000EEEFFAE0D5CFC080D180A7E7CA16DA0602
:1044800009F05ECEA895709160007861709360002D
:10449000B091D103B0936000EE3F2AE0F20791F0B3
:1044A0002091FE0A3091FF0A3183208349CEE080BB
:1044B000F180B7E7EB16FB0641F2F092FF0AE092BB
:1044C000FE0AC3CF1092FF0A1092FE0A39CE0E9454
:1044D0006F0AFC01028113810115110509F4E7CE71
:1044E000D801ED91FC910190F081E02DBE016B5E51
:1044F0007F4FC8010995811123CEF80100851185F0
:10450000EBCF181619060CF41BCED1CE11E0F11228
:10451000BDCE6CE77FE003CF0F920FB68F939F93D2
:10452000EF93FF938091C4038D5F8D3708F08D5713
:104530008093C403E5ECF3E080818E4F808391810A
:104540009F4F918382818F4F828383818F4F83839B
:10455000E9ECF3E080818F5F808381818F4F8183DD
:1045600082818F4F828383818F4F83838FB18F604E
:1045700066991C9B88278F3681F48091C303981B12
:10458000963068F0E0E0F8E087E78083818388E197
:1045900080936000F0936000FFCF9093C303FF917E
:1045A000EF919F918F910FBE0F9018951F920F92D0
:1045B0000FB60F9211242F933F934F935F936F93F6
:1045C0007F938F939F93AF93BF93EF93FF938091CC
:1045D000BA029091BB02A091BC02B091BD020097BB
:1045E000A105B10539F12091B902211105C0369A12
:1045F0003091B80231114F9A0197A109B109B7FD65
:1046000008C08093BA029093BB02A093BC02B093FF
:10461000BD02FF91EF91BF91AF919F918F917F91DB
:104620006F915F914F913F912F910F900FBE0F901F
:104630001F9018950E943E0CECCFEFEBF9E013822F
:10464000128288EE93E0A0E0B0E084839583A68395
:10465000B7838BE191E0918380838FEF9FEF958704
:1046600084878DEE99E090931E0A80931D0A80E066
:1046700090E890931C0A80931B0A46983E9A5F9894
:10468000579A0895CDB7DEB72F97DEBFCDBF789488
:1046900083E084BD83E085BD81E080936E00E1E826
:1046A000F0E083E08083E0E881E08083E1E983E07B
:1046B0008083E0E981E08083E1EC87E08083E3ECC4
:1046C00081E08083E0EC82E08083E2EC81E0808323
:1046D000EAE787E08083806880831092E20310928B
:1046E000D2031092D4030091D70001600093D70049
:1046F00010EA1093D80029B5206129BD39B5326080
:1047000039BD09B400FEFDCF81E090E00E94910B1D
:104710004091D8004F7C40614093D8005091E00018
:10472000507F5093E0006091E1006E7E6093E10065
:104730007DE07093E200559A209A91EC90937C0072
:10474000A1E7A5B9B7E6B4B9E5E3EBB9FFE3FAB978
:10475000769A6E9880EF81BB10BA00E50CBD11E02F
:104760001DBD85E00E94B10E599A85E00E94B10EF0
:104770005C98EDE1F5E025902EBC00000DB407FE3D
:10478000FDCFEA32C1F75C9A21E82093640031E062
:104790003093650080E80E94B40E8823A9F05C98ED
:1047A00045EA4EBD00000DB407FEFDCF5C9A2E9881
:1047B00058982D985091640050625093640061E0C5
:1047C00063BF889513BEFBCF84E00E94B40E88239C
:1047D000B9F12D9884E80E94B40E8823A1F02D9A97
:1047E00088EC0E94B10E58986FEF82E090E00E9432
:1047F000B83284EF91E00E94910B589A84E80E94AD
:10480000B40E8111FBCF84E10E94B40E8823A1F085
:104810002D9A88EC0E94B10E2E9860E082E090E024
:104820000E94B83284EF91E00E94910B2E9A84E1AD
:104830000E94B40E8111FBCF88EC0E94B10EC4CF50
:104840002D9A71E2709302011092BA039091E602E0
:1048500091709093E602A0910B03A170A0930B03BB
:10486000B0913003B170B09330031092CB0210922C
:10487000D2021092D9021092E00213EEA12E13E0A0
:10488000B12EF5018481887F84608483F8E0AF0EC7
:10489000B11C23EAA21624E0B20699F73FB6F894B9
:1048A0004090C5035090C6036090C7037090C80342
:1048B0003FBE4092BF035092C0036092C10370920A
:1048C000C2035FB6F8944091C5035091C60360914E
:1048D000C7037091C8035FBE6090BD037090BE03B4
:1048E000640E751E8090BF039090C003681879080D
:1048F0007092BE036092BD034093BF035093C00308
:104900006093C1037093C2037090C5039090C1027D
:10491000872D8919F82FC090C002CC2049F0109241
:10492000C00280E090E0892B61F20E940000C9CFB4
:10493000D09002018D1540F4FF5FFD1590F791E0D6
:1049400093BF889513BEEDCF01E00093C002709233
:10495000C102EEEBF2E08081918101968083918328
:104960001091BC032091BD033091BE03223231056A
:1049700014F40C94122E3091A7033F5F3093A703D9
:10498000113009F458C610F40C94622D123071F0F5
:10499000133011F40C94E12DE091BD03F091BE03AE
:1049A000B197F093BE03E093BD03DACF5091A30417
:1049B000552349F051505093A304511104C0109253
:1049C000A5041092A404E3DAE82E782F7170982FD2
:1049D000927084FF74C0272E2194992319F0F1E07E
:1049E0002F2E271AF12C0091BB048091B3040023D1
:1049F00009F470C001500093BB04A091B804AF1536
:104A00000CF0ADC0AF5FA093B8043090B804532C45
:104A100055948090B304580C5092B304E2FA772472
:104A200070F8E3FC7A942091C2023091C3022F5FA8
:104A30003F4F3093C3022093C202932C990C930CE6
:104A40004EE0249E900C1124892D711003C0C12CBE
:104A50002220A1F06AE0269FE02D1124F0E0EE0F65
:104A6000FF1FE15EFF4E2591349137FF02C02158B0
:104A70003F4F220F232F221F330BC22E5091B90418
:104A8000552379F051505093B9040E945A11837004
:104A900099270197C80E0E945A118F719927409744
:104AA000890D7091B70378170CF05EC07A5F709330
:104AB000B70387170CF060C08093B7035DC0F12C7B
:104AC000772311F0BAEFFB2E992311F0B6E0FB0E1D
:104AD000212C89CFE5FE91CFE091BD04E43108F4AB
:104AE0008CCF18E01093BB0426E02093B9044090CB
:104AF000AF045090B004805E0E945E182091B30411
:104B0000E0E2E20FF0E0EE0FFF1FE15EFF4E4591A5
:104B1000549157FF02C04D5F5F4F5595479555958E
:104B200047956090B1047090B204460D571DBC01CA
:104B300097FF02C06D5F7F4F759567957595679577
:104B4000640D751D8FEA94E00E94C10E3091BD0482
:104B500034513093BD048AE295E01ED94ECFFA1647
:104B60000CF053CFA1504FCF871734F47650709389
:104B7000B70378170CF4A0CF8091B8038C1544F4D8
:104B80008D5F8093B803C81654F4C092B80307C071
:104B9000C8162CF483508093B8038C15B4F380911D
:104BA000B3040E945E186C018091B304E82FF0E01A
:104BB000EE0FFF1FE15EFF4E45905490805C0E9417
:104BC0005E187C01E091B304E05CF0E0EE0FFF1FA3
:104BD000E15EFF4E05911491E72D770CFF0B4E9E81
:104BE000C0014F9E900D5E9E900D112448E1642EF1
:104BF000712CB3010E942B338090B6049090B704BF
:104C0000860E971E022C000C3308CE9EC001CF9E4C
:104C1000900DDE9E900D1124B3010E942B33E09184
:104C2000B404F091B504E60FF71FE29CC001E39CC9
:104C3000900DF29C900D1124B3010E942B33E60FCE
:104C4000F71FF093B504E093B404029DC001039DE7
:104C5000900D129D900D1124B3010E942B33860EEE
:104C6000971E9092B7048092B60497FE03C063E04B
:104C7000860E911C9594879495948794F7FD3396AE
:104C80006F01D594C794D594C7942091AF04309107
:104C9000B0042C0D3D1D3093B0042093AF04A091BF
:104CA000B104B091B204A80DB91DB093B204A093A1
:104CB000B104A6D8882371F14091B1045091B20497
:104CC000481959095093B2044093B10499D88823E4
:104CD00009F16091AF047091B0046C197D09709373
:104CE000B0046093AF048091B1049091B204880D38
:104CF000991D9093B2048093B10482D8882351F017
:104D00004090B1045090B204481859085092B2042F
:104D10004092B104E090B404F090B504B7E0BE9DB9
:104D2000F001BF9DF00D1124F7FD379603E0F595D6
:104D3000E7950A95E1F7F093B504E093B404009188
:104D4000B6041091B704F7E0F09FD001F19FB00DC9
:104D50001124B7FD179613E0B595A7951A95E1F7BD
:104D6000B093B704A093B6041091BD04143638F480
:104D7000D090BB04D11003C01F5F1093BD0490916D
:104D8000BA04992319F091509093BA048091AF041A
:104D90009091B00497FF02C081509F4FF92E00916F
:104DA000B1041091B20417FF02C001501F4F312E01
:104DB000612F8F2D0E941B0F863009F4DAC008F096
:104DC0009BC0853009F4B6C006EC12E0F80195816D
:104DD000992309F45CC19150958384810E945E18E7
:104DE00097FD03961C013594279435942794F80178
:104DF000E481F0E0EE0FFF1FE15EFF4E65907490DE
:104E000077FE03C0F3E06F0E711C75946794759480
:104E10006794D8018D909C901197820C931C8D9271
:104E20009C92F801C280D380C60CD71CD382C28268
:104E30003681EFEA4E2EE4E05E2E3F3F41F028E05F
:104E4000329F90011124A9014D515C4F2A01B601F6
:104E5000C4010E94310F882309F4CCC097FE03C01F
:104E60003FEF830E911CF92C492CD7FE03C04FEF66
:104E7000C40ED11C9D2C6D2D842D0E941B0F8930DA
:104E800009F0B5C040E06D2D842D0E94FE0EDA863B
:104E90001986C984DA8450E8C50ED11CFC861B86AD
:104EA000EB84FC8460E8E60EF11C41E0B601C7012A
:104EB0000E9475110E945A1165E070E00E9417333C
:104EC0008130910509F48BC008F483C0029709F47E
:104ED0008CC080E696E00E94CC1EF801628173814E
:104EE000661977098081918140E0821993090E94B7
:104EF0007511F8011582CBC0873009F452C0883093
:104F000009F062CF40E0612F8F2D0E94FE0E81EEEE
:104F10009FE00E94CC1E48EA55E05093A5044093C0
:104F2000A4047AE57093A3046091AD046F5F60936D
:104F3000AD044ACF3091BC04343608F045CF3C3440
:104F4000B0F034E63093BC0440E0632D8F2D0E9416
:104F5000FE0E81EE9FE00E94CC1E24EF35E03093E0
:104F6000A5042093A4045AE55093A3042DCF375EE3
:104F7000E9CF40E0612F8F2D0E94FE0E81EE9FE071
:104F80000E94CC1E0EED15E01093A5040093A4041E
:104F9000FAE5F093A304A091AE04AF5FA093AE0432
:104FA00013CF40E0612F8F2D0E94FE0E81EE9FE017
:104FB0000E94CC1E80EC95E09093A5048093A404FD
:104FC000BAE5B093A304E091AC04EF5FE093AC04C6
:104FD000FBCEA601B70183E00E943E157ACF45E0E3
:104FE000692D842D0E94FE0E74CF46E0F9CF8EE02D
:104FF00096E071CF8FEA481684E0580609F0A0C009
:1050000073EEE72E73E0F72EF7017481B72FB770B8
:10501000B430B1F120813181A90140565109841683
:10502000950674F1205A3F4F281539054CF18281BD
:1050300093819C0120563109C216D3060CF1805A87
:105040009F4F8C159D05E4F095819B3008F05BC067
:10505000EB2FF0E0EA55FB4FA181AF5FA183787F92
:105060007460F701748380E696E00E94CC1EF7011D
:105070006281738141E0808191810E9475112DCF01
:10508000F8E0EF0EF11CAE14BF0409F0BDCF095FCC
:105090001F4FF2E0023E1F0709F098CE22EE32E0E9
:1050A000F90114811E7FA9014B5D5F4F112309F4A3
:1050B00091C035964E175F0709F488C0A081A038CB
:1050C00001F183818D5F838372800A2F0A2E000C89
:1050D000110B070D111D77FC1A9501581F4F0F3F3B
:1050E000110568F46181082E000C990B860F911D43
:1050F00067FD9A9581386FEF96070CF058C0B0E8BD
:10510000B0833496D7CF9A5095838EE096E00E9474
:10511000CC1EF7013481377C3861532E3483C701AC
:105120000E942F150696FC0164916295660F660F2A
:10513000607CF52DFF738F2E862AF7018482CDCEF9
:105140006091AF047091B004CB018056910988162C
:1051500099060CF49CCF605A7F4F681579050CF4C2
:1051600096CFA091B104B091B204FD01E056F109CF
:10517000CE16DF060CF48BCFA05ABF4FAC15BD0581
:105180000CF485CFC2010E942F15009709F4A5CE1B
:105190000496FC0184910E94E01E9090BC04911042
:1051A0009CCEF201548157705093A60496CE80385D
:1051B000910524F0128213827FE77183D280DA0E88
:1051C000D08231802380320C31829BCFF9018481DF
:1051D000825084839A014155534009F061CF03EE18
:1051E00013E0F8013481532F5770543051F0432F9E
:1051F000407C99F17091A7037F703054772309F4B4
:1052000055C0085F1F4FF4E0033A1F0751F7809124
:10521000B1049091B20497FF02C081509F4F692F53
:105220008091AF049091B00497FF02C081509F4FCE
:10523000892F0E941B0F843041F4109103011A3012
:1052400009F0F4C184E00E94CF100091BC04011168
:10525000A3CB84E00E94CF109FCB232F26952695C9
:1052600026952770213021F140F0223011F02330B3
:1052700041F6377C3860F80119C02091B1043091B3
:10528000B2044091AF045091B00462817381808177
:1052900091810E94C70F882309F4B3CF88E997E072
:1052A0000E94CC1EF8013481377C38603483A9CF4A
:1052B00067805680662D852D0E94920F882EC8012A
:1052C0000E942F15811085C0252D30E03E832D834F
:1052D000D22ECC2430E8C30ED11C462D50E0588786
:1052E0004F83542E442450E8450E511CFC01339644
:1052F000249130E0EE24FF24E21AF30AD8016D90E5
:105300007C90B6016619770947016E157F052CF070
:105310004901621773070CF44B01F80122803380B6
:10532000C201821993098E159F052CF0790182170D
:1053300093070CF47C01680C791CD8016D927C9267
:105340002E0C3F1CF801338222826FEA74E0C80100
:105350000E949E14882309F4ACC0C8010E942F1536
:10536000FC013796D490D11025C00496FC0184919D
:105370000E94E01E3090BC04311005C0F801B481D9
:10538000B770B093A604F8015481577C552E6894E9
:1053900054F85482C8010E942F150596FC013491DF
:1053A0003295330F330F307C652D6F73662E632A71
:1053B000F8016482D8012D903C9011972818390883
:1053C0002D923C92F801828093808E189F089382E0
:1053D0008282C8010E94D01460E1E62E882339F051
:1053E000682F70E080E190E00E942B33E62EC80128
:1053F0000E942F150796FC018491882309F401CFA0
:105400000E945A116E2D70E08617170608F0F9CE2B
:10541000E090B104F090B204C090AF04D090B0041A
:10542000F80142805380608071809701A601B2012B
:10543000C3010E94C70F882309F4E3CEC618D7081A
:10544000D7FE03C0FFEFCF0ED11C2D2DE418F508B9
:10545000F7FE03C03FEFE30EF11C8F2D2111C5C0F5
:1054600060ECF7FC04C060E4FF2009F4CACEC80178
:105470000E94C314882309F4C4CE8EE397E00E94EF
:10548000CC1EF8014481477CC42E6894C4F8C482C1
:10549000C8010E942F150596FC0124912295220F28
:1054A000220F207C9C2D9F73F92EF22AF801F482A2
:1054B000A8CEC614D70409F08CCF4214530409F0C7
:1054C00088CF4091AF045091B00457FF02C04150C3
:1054D0005F4FE52EFF24E7FCFA94CD80DE80EC18C8
:1054E000FD081E141F041CF4EE24E394F12CF7FEB7
:1054F00003C0EE24EA94FE2C9E2C4090B104509000
:10550000B20457FE03C03FEF430E511CC52CDD24EF
:10551000C7FCDA942F813885C21AD30A1C141D04E3
:105520001CF4CC24C394D12CD7FE03C0CC24CA9441
:10553000DC2C7C2C0E945A11F82EC8010E942F15D9
:105540000796FC019491992341F0C8010E94D01460
:10555000833018F49E2C91947194911039C07FE39C
:1055600099249A947F1528F49F2C9094991C99243F
:10557000991CF8014781470D6681690DC8010E9499
:10558000F114811126CFF8016681690D4781C801A8
:105590000E94F11481111DCFF8014781470D6681EA
:1055A000C8010E94F114811114CFF8014781470D01
:1055B00066816919C8010E94F11481110ACFF801AE
:1055C000478147196681690DC8010E94F11401CF16
:1055D0007110CFCFFFE377247A94FF1550F67F2C1C
:1055E0007094771C7724771CC4CFF11005C060E855
:1055F00027FD3DCF60E03BCF2F1106C060E21216C1
:105600000CF435CF60EA33CF992781950CF490954F
:10561000422F022E000C550B4817590709F0F1CD07
:1056200060EE12160CF423CF60E621CF1F5F1093BB
:10563000030181E008CEE091BA03F091BB03EE31A3
:10564000F10528F43196F093BB03E093BA0300917F
:10565000BA031091BB030E31110509F09DC90E94D8
:10566000C71F811199C97091E60271707093E602AB
:1056700010910B03117010930B03F0913003F17034
:10568000F09330031092CB021092D2021092D90202
:105690001092E002E3EEF3E0B481B87FB460B4832B
:1056A000389624E0E33AF207B9F710E000E0F12C75
:1056B000E12C4DE00BC001151105D9F33FE1E316D4
:1056C000F104B9F307311105A1F340E0602F8E2DED
:1056D0000E94FE0E4FEFE41AF40A50E2E516F104C0
:1056E00051F70F5F1F4F0831110509F7E12C00E05A
:1056F00026E14EE161E081E00E94D11100E0C12C81
:10570000D12CFF24F394E12C10E0212C50E0211641
:10571000E0F4512C552341F051E01BC051111CC045
:10572000212CF5CF81110FC0652D6E0D822D8F0DAF
:105730000E941B0F53941511F5CF51E0811101C048
:1057400050E02394E4CF51E0FCCF511102C0011787
:10575000A0F11F5F183111F7E39437E1E312D4CFC2
:10576000F3946FE1F612CFCF073050F112E0A02F83
:10577000A250BB0B1A171B060CF6412E4D0C4DE028
:1057800062E06C0D842D0E94FE0E612E6C0C4DE0CB
:10579000662D82E08D0D0E94FE0E6C2D600F635011
:1057A0004DE0842D0E94FE0E4DE0662D8D2D800F64
:1057B00083500E94FE0E1F5FDACF012F6701C9CF11
:1057C00050E4852E1FEF0E945A11082F0F710E947E
:1057D0005A1168E170E02BD7E82E682F802F0E94C5
:1057E0001B0F811114C06E2D802F0E94990F9130D4
:1057F00071F442E06E2D802F0E943A0F843038F011
:1058000042E06E2D802F0E94FE0E8A941FEF1150F1
:1058100011F08110D8CF48E1442E1FEF0E945A1199
:10582000082F0F710E945A1168E170E000D7682EAE
:10583000682F802F0E941B0F811128C06E861D8645
:105840006D857E8560587F4F802F90E0982F882748
:1058500020E831E040E851E080589F4F0E94C70F98
:10586000811114C0662D802F0E94990F91110EC0D6
:1058700041E0662D802F0E943A0F843038F041E0DD
:10588000662D802F0E94FE0E4A941FEF115011F0DA
:105890004110C4CF0FEF1FEF0E945A118F71C82E15
:1058A0000E945A1168E170E0C2D6F82E682F8C2D44
:1058B0000E941B0F811129C06F2D8C2D0E94990F02
:1058C00081FB992490F882FB772470F883FBDD2418
:1058D000D0F89230D1F4A82FA17080FF12C0992087
:1058E00009F44BC049E06F2D8C2D0E943A0F843093
:1058F00060F049E06F2D8C2D0E94FE0E01501FEFCD
:1059000004C09920D1F17110EDCF115011F00111A7
:10591000C3CF43E061E081E00E94FE0E44E065E118
:105920008DE10E94FE0E80910301813029F44CE04C
:1059300062E082E00E94FE0E28E0822E0FEF1FEF51
:105940000E945A118F71382E0E945A1168E170E03E
:105950006ED6582E0E945A1165E070E068D68230EB
:10596000910509F4A7C008F06CC0F6E02F2E01974E
:1059700009F471C095E0292E6EC0772019F0DD2062
:1059800021F2B0CFDD2009F4C0CFAA2309F4BDCFA6
:10599000A9CF8110D5CF00E810E0E12C682D8E2D25
:1059A0000E941B0F813009F088C00E945A116E2D91
:1059B00070E0762F662760587F4FA80183700E94A1
:1059C0003E1540E0682D8E2D0E94FE0E83941395A7
:1059D0000038E8E11E0709F720E831E03093B00411
:1059E0002093AF043093B2042093B10490E29093DB
:1059F000B30474E67093BD041092BA041092B90413
:105A00001092BB041092B5041092B4041092B70423
:105A10001092B6041092B804FFB7F8946091C503D1
:105A20007091C6038091C7039091C803FFBF609334
:105A3000BF037093C0038093C1039093C20382E0BD
:105A400009CCB7E02B2E8330910529F0A8E02A2E4F
:105A5000049709F08FCF652D832D0E941B0F8111B4
:105A600023C0652D832D0E94990F9130E9F4422DBA
:105A7000652D832D0E943A0F8430B0F043E0652DF0
:105A8000832D0E943A0F873078F044E0652D832DF6
:105A90000E943A0F873040F0422D652D832D0E94E1
:105AA000FE0E8A940FEF10E00150110909F071CF3A
:105AB000812C71CF8AE0282ECECFE39440E2E4120D
:105AC0006DCF84CF0E945A110E94C71F83FF0BC065
:105AD0009090C40293FC07C0B1E0F091BA03F111B9
:105AE000B0E0B093BA030E94C71F82FF0BC0709052
:105AF000C40272FC07C051E0D090BA03D11050E04C
:105B00005093BA030E94C71F807359F03091C402AA
:105B1000307339F46091BA03662349F0613009F4B7
:105B200042C00E94C71F8093C4020C94CC24A1E001
:105B3000A093030184E08093A6041092AB0410921A
:105B4000AE041092AC041092AD041092A70410920F
:105B5000A8041092A9041092AA0440E851E05093BE
:105B6000B0044093AF045093B2044093B10420E2D8
:105B70002093B30494E69093BD041092BA0410925B
:105B8000B9041092BB041092B5041092B4041092A0
:105B9000B7041092B6041092B8049093BC0481E04C
:105BA0000E94CF10BECF3090C502311005C03E9A82
:105BB000579A6093C502B5CF1092C5023E98579888
:105BC000B0CFA091BA03B091BB03AE31B10528F4B8
:105BD0001196B093BB03A093BA034091BA035091BE
:105BE000BB034E31510579F40E94C71F807359F0F1
:105BF0008091BA039091BB0301969093BB0380936D
:105C0000BA030C94CC246091BA037091BB036F313A
:105C1000710511F00C94CC240E94C71F81110C94C3
:105C2000CC2418CB123009F4BBC0B8F4112309F40A
:105C300056C0113009F4A3C0EFEBF5E0812CA0E0D1
:105C4000B8E000800EBC8110012C1197A0FDFDCFA3
:105C50000192B9F70DB40C949124133009F450C398
:105C6000143051F7A091BA03B091BB03AB2B31F4C0
:105C700081E090E09093BB038093BA030FEF10E0B4
:105C80002091BA033091BB031901369427943092C6
:105C9000BB032092BA0320FF08C0FEE62F26FFE1D7
:105CA0003F263092BB032092BA038091BA039091B1
:105CB000BB03BC01660F672F661F770B719540E031
:105CC0008F770E946A184091BA035091BB0341300C
:105CD000510509F048C483E00E94CF10ADCF0E9467
:105CE000F00921E042E162E081E199E00E9438118F
:105CF00021E040E267E080E099E00E94381121E075
:105D000048E164E08AEF98E00E94381121E048E120
:105D100065E083EF98E00E943811B091C50221E060
:105D200044E365E0BB2341F180EF98E00E94381125
:105D30006091BA036C5F21E040E18AEE98E00E9436
:105D400038115091A7037AEAC72E78E0D72E52FD7A
:105D500004C06AE6C62E68E0D62EE12C0FEF29E0DB
:105D60004AE060E0C6010E947E1E29E04AE06EE63D
:105D7000C6010E947E1E60CF8CEE98E0D7CF0E94B5
:105D8000F00921E04EE163E089E299E00E943811D8
:105D9000809103014AE563E090E00E94F9104CCF46
:105DA000C090AF04D090B004D092A903C092A803D1
:105DB000E090B104F090B204F092AB03E092AA0339
:105DC0005090B3045092AC039091A6039F5F9093C0
:105DD000A6035FEB852E55E0952E4FEB57E0F401BF
:105DE0004E175F0741F035E5308311822AEA22839E
:105DF00013823496F5CF31E8315049F005E5008340
:105E00006FEF61835AEA528363833496F5CF109221
:105E1000BE041092A5038091B7035091B803505E61
:105E2000AFE3B5E0082E000C990B9C0146E0220F71
:105E3000331F4A95E1F7EFEBF4E040E01D92152F98
:105E4000130F11934F5F281B390B4038B9F7C60168
:105E5000D7FE02C081509F4F9093B503C701F7FE54
:105E600002C081509F4F9093B603752C7194872D7B
:105E70000E945E188C019093AE038093AD03E72DD2
:105E8000F0E0EE0FFF1FE15EFF4E659074907092A0
:105E9000B0036092AF0380E2382E3518832D0E9444
:105EA0005E189093B2038093B103E32DF0E0EE0F00
:105EB000FF1FE15EFF4E259134913093B403209390
:105EC000B303852D0E945E18E52DF0E0EE0FFF1F55
:105ED000E15EFF4E4590549077E0789FA001799F56
:105EE000500D11244C0D5D1D749DC001759D900DCC
:105EF00011248E0D9F1D38EFF32EF90EF8EFF50FDC
:105F0000F7FDF0E0F7FCF12CEF2E60E16F1714F4D1
:105F1000F0E1EF2EB8E0BF1514F4E8E0FE2E70E1DA
:105F2000572E5E0CDD24D394101611063CF0552438
:105F30005A945E0C5FE0E50EDD24DA9460E1C62E33
:105F4000CF0C2224239477FC07C0CC24CA94CF0C16
:105F5000AFE0FA0E22242A9417FF03C01195019591
:105F6000110977FE03C07194619471080615170535
:105F700074F4CF14B9F07E2C571431F06F2D872DA7
:105F80000E947D1C7D0CF8CFF20CF3CFED0C5E145B
:105F900049F01F2DC116D1F3612F8E2D0E947D1C5B
:105FA000120DF8CF53EE452E53E0552EF2014481E9
:105FB000942F9770943089F1342F36953695369515
:105FC0003770E12C333029F4F091A6030F2F0170C4
:105FD000E02E4770423011F0313039F48091A70340
:105FE00040E2642E712C83FF02C0712C612CC2012F
:105FF0000E942F15FC013996049131972491FC01E0
:1060000085919491F2014281538160817181660C86
:10601000771C860D971D0E94F717F8E04F0E511C54
:10602000A414B50409F0C2CF96ECC92E92E0D92E83
:1060300022EE622E22E0722EF6013580332079F0B6
:10604000428153816081718126812F3F09F059C0BF
:1060500088E799E0E12C02E020E20E94F717F7E0E0
:10606000CF0ED11C6C147D0439F702EE12E081E5ED
:10607000E82E83E0F82EF80174817E7FE9F06281DA
:1060800073819E012F5F3F4FAE014D5F5F4F808157
:1060900091810E94AB17882379F089810E945D1558
:1060A000FC01892B49F0628161606283BB81B3830B
:1060B00059805682118300830B5D1F4FE016F10655
:1060C000D1F6512CF090A5035F1408F090C057E072
:1060D000559ED0011124FD01EF5AFC4F8081918122
:1060E00006816381D280D0FC0FC0AD5ABC4F2C908A
:1060F00021FAEE24E0F8258144810E947E1E53940B
:10610000E1CF88E399E0A6CF202E312CC62E660F72
:10611000DD08A101440F551F5E834D839601D7FE14
:1061200002C030E020E021543B4FD9011C911F8771
:10613000FC01748070FA442440F89C012B5D3F4FB1
:1061400038872F838C010B5F1F4F8F8198858017B5
:106150009107A9F2D8013C91303809F445C06D810E
:106160007E8136033001379F700C1124E72CFF2409
:10617000E7FCFA94EC0CFD1CF801518156039001E8
:10618000579F300D1124632E772467FC7A949F85E6
:10619000690E711C97FD7A942FE7E216F10420F541
:1061A0003FE36316710400F5D701A15CBA4FFC917F
:1061B000F215130409F0C4F4442D662D8E2D0E94AF
:1061C0006A18FF24F394FE0C442D662D8F2D0E9437
:1061D0006A186394442D662D8F2D0E946A18442DF1
:1061E000662D8E2D0E946A180C5F1F4FAECF8091D6
:1061F000B70387FD8D5F85958595082E000C990B5B
:10620000AC014A5A5F4F2091B803022E000C330BA9
:106210006BE270E0621B730BE091BB04EE2309F4A8
:106220005CC0BBEAEB9F812D1124869590E0EAE9E2
:10623000FAE00491EBE9FAE0E490681B790B615015
:1062400071096A01C81AD90AC601E3E0CE2E30E00E
:1062500020E04CE95AE001970E94E30C4091BC0415
:1062600064E87BE08FE399E00E94FD094091BD0462
:106270006CE77BE08FEB98E00E94FD093090BA0458
:106280003320F1F04DE356E0F40171817E7F71839C
:10629000EF57FC4F10811F771083FFEF8F1A9F0A73
:1062A0004815590589F7EFEBF5E01082DF01A15899
:1062B000BF4F1C92E058FF4F29E0EF3BF207A9F7D0
:1062C0008091A4049091A504009709F4B5CC20E036
:1062D00040E060E00E943811AFCCE8EBF9E00491B7
:1062E000E9EBF9E0E4906DE270E0621B730B53E0C0
:1062F000C52E30E020E04AEB59E0885A9F4FACCFE2
:106300000E94F00921E04EE260E08CE29FE00E94F2
:106310003811C09003013091A604D12C323009F419
:1063200013C108F0EEC0332309F405C1313009F47C
:10633000F5C021E044E162E080EA9EE00E9438116D
:10634000E12C0FEF29E045E160E080E69EE00E944D
:106350007E1E8091AB0442E164E090E00E94F9105F
:1063600029E046E260E080E29EE00E947E1E80918D
:10637000AC0442E166E090E00E94F91029E045E1BA
:106380006EE180EE9DE00E947E1E8091AD0440E3B0
:1063900064E090E00E94F91029E046E26EE180EAB4
:1063A0009DE00E947E1E8091AE0440E366E090E096
:1063B0000E94F910F090A70300E210E0F3FE02C083
:1063C00010E000E021E044E562E089E99DE00E9400
:1063D00038114801880C991CE12C0FEF29E045E1A8
:1063E00062E4C401875E924F0E947E1E8091A704E2
:1063F00044E564E090E00E94F91029E046E262E49E
:10640000C4018756934F0E947E1E8091A80444E5E4
:1064100066E090E00E94F910EE24E39429E045E163
:1064200060E6C401875E934F0E947E1E8091A9049E
:1064300042E764E090E00E94F910E12C29E046E296
:1064400060E6C4018756944F0E947E1E8091AA0484
:1064500042E766E090E00E94F91031E0C31AD108EB
:1064600014E11C9DC0011D9D900D11242091A604D6
:10647000243011F48C509E4F9090AB047090AC047B
:106480007AE0779E70011124FFE09F9EE00CF11CE2
:106490001124D090AD0468E0D69EF0011124EE0ED8
:1064A000FF1E3090AE04B4E03B9E20011124E40CAA
:1064B000F51C5090A704579EE00CF11C112460902D
:1064C000A804679EE00CF11C11245091A904A5E0DA
:1064D0005A9FE00CF11C1124C090AA0404E0C09E55
:1064E00010011124E20CF31CE80EF91E21E044E136
:1064F00067E08CE89BE00E94381148E467E0C70140
:106500004CCC333051F1343009F013CF21E04CE062
:1065100061E081E19FE00E9438110BCF21E048E06B
:1065200061E087EF9EE00E94381140E761E0C6011C
:106530000E94F910FECE21E044E061E08BED9EE088
:106540000E94381144E7F2CF21E04AE061E082EC9A
:106550009EE00E9438114EE6E9CF21E044E061E080
:1065600086EA9EE0EDCF0150110909F089CB64CB9A
:10657000262FF999FECF92BD81BDF89A019700B4FC
:10658000021639F01FBA20BD0FB6F894FA9AF99A9C
:106590000FBE0895052E97FB16F400940FD057FDFB
:1065A00005D014D007FC02D046F408C050954095A1
:1065B000309521953F4F4F4F5F4F089590958095AF
:1065C000709561957F4F8F4F9F4F0895A1E21A2ECE
:1065D000AA1BBB1BFD010DC0AA1FBB1FEE1FFF1F87
:1065E000A217B307E407F50720F0A21BB30BE40BD7
:1065F000F50B661F771F881F991F1A9469F760951E
:106600007095809590959B01AC01BD01CF010895D7
:10661000A29FB001B39FC001A39F700D811D1124E3
:10662000911DB29F700D811D1124911D0895AA1B0B
:10663000BB1B51E107C0AA1FBB1FA617B70710F06D
:10664000A61BB70B881F991F5A95A9F7809590959F
:10665000BC01CD01089597FB072E16F4009406D0D7
:1066600077FD08D0E4DF07FC05D03EF490958195D6
:106670009F4F0895709561957F4F0895EE0FFF1F0E
:106680000590F491E02D0994C3DF332312F48A1BA3
:106690009B0B01C0BDDFB7FF0895821B930B0895CC
:1066A0002F923F924F925F926F927F928F929F9222
:1066B000AF92BF92CF92DF92EF92FF920F931F9310
:1066C000CF93DF93CDB7DEB7CA1BDB0B0FB6F894C1
:1066D000DEBF0FBECDBF09942A88398848885F8401
:1066E0006E847D848C849B84AA84B984C884DF8072
:1066F000EE80FD800C811B81AA81B981CE0FD11D56
:106700000FB6F894DEBF0FBECDBFED010895F8942B
:02671000FFCFB9
:1067120001001001FFFFFFFF00E100000000000088
:1067220000C1808100000000000000830AA30BA5C5
:0A6732000A9A0AC30AA80AB40A0072
:00000001FF
